:020000040000FA
:061000001FEF3CF012009E
:06100800B9EF26F0120012
:0610180022EF08F01200B7
:06102A0002008C780000BA
:1010300099010000640000008A780000B80E0000EA
:0410400002000000AA
:0C104400D8CFE4FFE0CFE4FFE46EDACF89
:10105000E4FFE2CFDAFFE9CFE4FFEACFE4FFF3CF2A
:10106000E4FFF4CFE4FFE652D9CFE6FFE1CFD9FFAA
:10107000040EE126020EDB6A030EDB6AA4A67ED311
:10108000A4960501FE5101E1A1D0030E526E2D5030
:10109000EA6A510FE96E010EEA22EF50525C30E12C
:1010A0002D50E96EEA6AD890E936EA36690EE926EB
:1010B000010EEA22EECF52F0EFCF53F053C052F0C0
:1010C000536A5250D76E2D50E96EEA6AD890E936CD
:1010D000EA36690EE926010EEA22EECF52F0EFCF92
:1010E00053F05250D66EF28AF294D58E2D50EA6AA1
:1010F000510FE96E010EEA22040EEF6E2D502F6E95
:10110000020E526E2E50EA6A510FE96E010EEA226B
:10111000EF50525C49E12E50E96EEA6AD890E93608
:10112000EA36690EE926010EEA22EE50ED1009E1D9
:101130002E50EA6A510FE96E010EEA22010EEF6E9F
:1011400033D0080E2E5C0CE2070E2E14526E010EE8
:10115000525204E0E846FE0B5206FCE189121AD016
:10116000100E2E5C0CE2070E2E14526E010E52521F
:1011700004E0E846FE0B5206FCE18A120BD0070E93
:101180002E14526E010E525204E0E846FE0B520637
:10119000FCE18B122E50EA6A510FE96E010EEA2231
:1011A000030EEF6E2E502D6E2E2A060E2E5C02E1DF
:1011B000080E04D0130E2E5C03E1160E2E6E59D1CC
:1011C000180E2E5C01E055D12E6A53D10E0100514C
:1011D00001E14FD10E01012B0E01AC510E01015D59
:1011E00001E247D1016B0E01AA51EA6A320FE96EA2
:1011F0000E0EEA22EF500E01EA6AAD25E96EAE51FD
:10120000EA22EF6A79907B6A7A6A0E01AA2B0E01B4
:10121000AB510E01AA5D01E3AA6BAA51E96EEA6A1D
:10122000D890E936EA36020EE9260E0EEA22EE5092
:10123000ED1001E11ED1AA51E96EEA6AD890E936B3
:10124000EA364A0EE9260E0EEA22EECF52F0EFCF32
:1012500053F0AA51E96EEA6AD890E936EA36020EEE
:10126000E9260E0EEA22EECF54F0EFCF55F054509F
:10127000521802E15550531801E1BDD0AA51E96E50
:10128000EA6AD890E936EA364A0EE9260E0EEA22D4
:10129000EECF54F0EFCF55F0AA51E96EEA6AD8903C
:1012A000E936EA36020EE9260E0EEA22EE50545CCA
:1012B000526EEE505558536E020E52C0DBFF030EB5
:1012C00053C0DBFF020EDBCF52F0030EDBCF53F037
:1012D00053343BE252500008000E535436E2020EE3
:1012E000DBCF52F0030EDBCF53F0AA51E96EEA6A6E
:1012F000D890E936EA367A0EE9260E0EEA22EECFCB
:1013000054F0EFCF55F05250545C5350555857E2BB
:10131000AA51E96EEA6AD890E936EA367A0EE926E9
:101320000E0EEA22EECF52F0EFCF53F0AA51E96E43
:10133000EA6AD890E936EA36020EE9260E0EEA226B
:101340005250EE265350ED2256D0020EDBCF52F013
:10135000030EDBCF53F0526C531E000E5322AA51E2
:10136000E96EEA6AD890E936EA367A0EE9260E0E78
:10137000EA22EECF54F0EFCF55F05250545C535068
:1013800055581DE2AA51E96EEA6AD890E936EA3664
:101390007A0EE9260E0EEA22EECF52F0EFCF53F08E
:1013A000AA51E96EEA6AD890E936EA36020EE926D1
:1013B0000E0EEA225250EE5E5350ED5A1CD0AA5146
:1013C000E96EEA6AD890E936EA364A0EE9260E0E48
:1013D000EA22EECF52F0EFCF53F0AA51E96EEA6A5B
:1013E000D890E936EA36020EE9260E0EEA2252C0FD
:1013F000EEFF53C0EDFFAA51EA6A320FE96E0E0EFE
:10140000EA22EF500E01EA6AAD25E96EAE51EA22FA
:10141000120EEF6EF29E0E01AA51E96EEA6AD890A2
:10142000E936EA36020EE9260E0EEA22EECF52F037
:10143000EFCF53F053C052F0536A5250B66EAA51D8
:10144000E96EEA6AD890E936EA36020EE9260E0E0F
:10145000EA22EECF52F0EFCF53F05250B56EF00EBD
:10146000B4140009B46EF00EB4140909B46E798096
:10147000F28E000ED8802154000E22542EE2302A23
:10148000000E31222150305C2250315826E3306A60
:10149000316A030E255C1FE22350EA6A480FE96EA9
:1014A000010EEA2280CFEFFF2350EA6A4B0FE96E6C
:1014B000010EEA2281CFEFFF2350EA6A4E0FE96E58
:1014C000010EEA2282CFEFFF232A030E235C01E301
:1014D000236A252A02D0216A226A000ED880265467
:1014E000000E275419E22B50000816E2322A000E93
:1014F00033222650325C275033580EE3326A336A67
:10150000030E2A5C07E2282A030E285C01E3286AFE
:101510002A2A02D0266A276A2B5000080AE2346A77
:101520003450040DF328C26E9E9C9F9C9D8CC280FB
:10153000C2820101995101E11DD1DE6ADD6ADECF6F
:1015400052F0DDCF53F0040E525C000E535801E30D
:1015500011D1DECFE9FFDDCFEAFF010ED890E936E9
:10156000EA36E806FBE19A0EE926010EEA22EE5081
:10157000ED1001E1D3D0DECFE9FFDDCFEAFF010EB0
:10158000D890E936EA36E806FBE1AA0EE926010E14
:10159000EA22EE50ED1026E1D9CFE9FFDACFEAFFDB
:1015A000EE50ED1001E18180D9CFE9FFDACFEAFFFB
:1015B000010EEE1803E1ED5001E18182D9CFE9FF80
:1015C000DACFEAFF020EEE1803E1ED5001E181846B
:1015D000D9CFE9FFDACFEAFF030EEE1803E1ED50B1
:1015E00001E18186DECFE9FFDDCFEAFF010ED89071
:1015F000E936EA36E806FBE1AA0EE926010EEA2200
:10160000EECF52F0EFCF53F0DECFE9FFDDCFEAFFB0
:10161000010ED890E936EA36E806FBE19A0EE92693
:10162000010EEA22EECF54F0EFCF55F0545052188D
:1016300029E15550531826E1D9CFE9FFDACFEAFF67
:10164000EE50ED1001E18190D9CFE9FFDACFEAFF4A
:10165000010EEE1803E1ED5001E18192D9CFE9FFCF
:10166000DACFEAFF020EEE1803E1ED5001E18194BA
:10167000D9CFE9FFDACFEAFF030EEE1803E1ED5010
:1016800001E18196DECFE9FFDDCFEAFF010ED890C0
:10169000E936EA36E806FBE1AA0EE926010EEA225F
:1016A000EE2A000EEF22DECFE9FFDDCFEAFF010ECA
:1016B000D890E936EA36E806FBE1AA0EE926010EE3
:1016C000EA22EECF52F0EFCF53F0DECFE9FFDDCFCD
:1016D000EAFF010ED890E936EA36E806FBE1A20EF1
:1016E000E926010EEA22EECF54F0EFCF55F0545028
:1016F00052183AE15550531837E1DECFE9FFDDCFFC
:10170000EAFF010ED890E936EA36E806FBE1AA0EB8
:10171000E926010EEA22EE6AED6A26D0D9CFE9FF6A
:10172000DACFEAFFEE50ED1001E18190D9CFE9FF69
:10173000DACFEAFF010EEE1803E1ED5001E18192EC
:10174000D9CFE9FFDACFEAFF020EEE1803E1ED5040
:1017500001E18194D9CFE9FFDACFEAFF030EEE1859
:1017600003E1ED5001E18196DF2A010E01E2E7D6A7
:10177000DB2AE5D60201AB5101E0AB079EAC2CD0D1
:101780009E9CC450566E576E566AC3500001561048
:10179000546E57C055F03450060DF3CF52F0F4CFCD
:1017A00053F0000E5226010E53222850020D5250C3
:1017B000F324E96E5350F420EA6E54C0EEFF55C096
:1017C000EDFF342A2B50345C02E39D9C05D034504D
:1017D000040DF328C26EC282F2A442D0D59EF294C8
:1017E000F29A040E526E2F50EA6A510FE96E010E02
:1017F000EA22EF50525C34E1080E2F5C0DE2070E36
:101800002F14526E010E525204E0E846FE0B5206AF
:10181000FCE1E81C89161CD0100E2F5C0DE2070EAF
:101820002F14526E010E525204E0E846FE0B52068F
:10183000FCE1E81C8A160CD0070E2F14526E010E24
:10184000525204E0E846FE0B5206FCE1E81C8B16FF
:101850002F50EA6A510FE96E010EEA22020EEF6E76
:10186000040EE15C02E2E16AE552E16EE552E7CF87
:10187000D9FFE552E5CFF4FFE5CFF3FFE5CFEAFF6F
:10188000E5CFE9FFE5CFDAFFE550E5CFE0FFE5CFB3
:10189000D8FF1000D9CFE6FFE1CFD9FF020EE12635
:1018A000896A92682B6A8A6A93688B6A94688C96B4
:1018B0008C9495969594928E0501010EFD6F0E0104
:1018C000B869B969296A286A2A6A246A236A256A72
:1018D000216A226A266A276A306A316A326A336A62
:1018E000346A76827680769C769A76887696FA0E38
:1018F000776EDF6ADFCF49F00C0EE76E4918E8AE6D
:1019000002D0E73402D0E750495C36E2010EDB6AD0
:10191000DBCF49F0030EE76E4918E8AE02D0E7349A
:1019200002D0E750495C26E2DFCF49F04A6A49BE5F
:101930004A68060E4A02F3CF4AF04902F3CF49F053
:10194000F4504A26000E4926010E4A22010EDBCF32
:101950004BF04C6A4BBE4C68D8904B364C364950D5
:101960004B24E96E4A504C20EA6EEE6AED6A010E95
:10197000DB2ACED7DF2ABED70501F76BF86BF56BF4
:10198000F66BF96BFA6BFB6BFC6B2D6A2E6A2F6A98
:10199000DF6ADFCF49F0180EE76E4918E8AE02D0D3
:1019A000E73402D0E750495C1BE2DFCFE9FFEA6A87
:1019B000E9BEEA68D890E936EA36690EE926010EF2
:1019C000EA22EE6AED6ADFCFE9FFEA6AE9BEEA6879
:1019D000510EE926010EEA22010EEF6EDF2AD9D759
:1019E000D586D59AD59CF294F29AF194D08E7694BD
:1019F000A386A59642EC28F0C5EC36F0F28EF28C68
:101A00007684020EE15C02E2E16AE552E16EE552A3
:101A1000E7CFD9FF1200D9CFE6FFE1CFD9FF050EFE
:101A2000E126020EDB6A030EDB6A040EDB6A1CECA5
:101A30001DF02550000809E200EC14F0242A030EE2
:101A4000245C01E1246A2506F4D72A50000809E243
:101A500030EC14F0292A030E295C01E1296A2A06D8
:101A6000F4D7200E0501E76EA819E8AE02D0E734DE
:101A700002D0E750A85D01E2B7D16550020B01E04A
:101A8000B3D1400EE66E400EE66E020EE66E28EC16
:101A900035F0E552E552E552E76E030EE7CFDBFF86
:101AA000DB50000801E324D1040EDB6A030EDB5097
:101AB000F36E040EDBCFF4FFF350F45C01E318D1B6
:101AC000040EDB50EA6A400FE96E020EEA22EFCF05
:101AD000DFFF0101F65141E10D0E496EDF50495C17
:101AE00005E00A0E4A6EDF504A5C37E1010EF66FE0
:101AF0000501F751EA6A000FE96E030EEA220D0EA6
:101B0000EF6EF72B010EDB6AF751F36E010EDBCFA0
:101B1000F4FFF350F45C1CE2010EDBCFE9FFEA6A4C
:101B2000E9BEEA68000EE926030EEA22EF50E66EEF
:101B3000010EDBCFE9FFEA6AE9BEEA68B20EE926E8
:101B4000010EEA22E552E750EF6E010EDB2ADCD7E8
:101B5000D5D90501F76BF86BBBD01B0EDF5C09E133
:101B6000F25107E1010EF26F1B0EF36FF46BF56B90
:101B7000AFD0F2050BE15B0EDF5C08E11B0EF35DFD
:101B800005E1F45103E15B0EF46FA2D0F20566E1CA
:101B9000410EDF5C63E11B0EF35D60E15B0EF45D03
:101BA0005DE1F36BF46BF56BF26B010EDB6ADBCF7F
:101BB000E9FFEA6AE9BEEA68000EE926030EEA22B6
:101BC000EF500D081CE0010EDBCFE9FFEA6AE9BE29
:101BD000EA68B20EE926010EEA22EF50E66E010E27
:101BE000DBCFE9FFEA6AE9BEEA68000EE926030EE8
:101BF000EA22E552E750EF6E010EDB2AD8D7010E3C
:101C0000DBCFF7F50501F751EA6A000FE96E030E25
:101C1000EA22EF6A1F0E496E720E4A6E4B6A49C085
:101C2000E6FFE66E4BC0E6FF56EC3AF0E552E552B1
:101C3000E552000EE66E030EE66E1C0E496E720E45
:101C40004A6E4B6A49C0E6FFE66E4BC0E6FF56ECB3
:101C50003AF04C6E050EE15E4C503AD0080EDF5C57
:101C60001CE10501F751000818E2F707F751EA6A8D
:101C7000000FE96E030EEA22EF6A190E496E720E2A
:101C80004A6E4B6A49C0E6FFE66E4BC0E6FF56EC73
:101C90003AF0E552E552E5521BD00D0EDF5C18E03C
:101CA0000A0EDF5C15E0200EDF5C12E30101F36B2E
:101CB000F46BF56BF26B0501F751EA6A000FE96E00
:101CC000030EEA22DFCFEFFF0101F66B0501F72BD0
:101CD0000501F751496E4A6A000E491806E1010EE6
:101CE0004A1803E12C86F76BF86B040EDB2ADED66C
:101CF0002C5001E178D02CA00FD0130E496E720E3B
:101D00004A6E4B6A49C0E6FFE66E4BC0E6FF56ECF2
:101D10003AF0E552E552E5522CA20FD0F40E496E8E
:101D2000710E4A6E4B6A49C0E6FFE66E4BC0E6FF95
:101D300056EC3AF0E552E552E5522CA40FD0D80EFD
:101D4000496E710E4A6E4B6A49C0E6FFE66E4BC0A3
:101D5000E6FF56EC3AF0E552E552E5522CA60FD0DC
:101D6000BC0E496E710E4A6E4B6A49C0E6FFE66EC4
:101D70004BC0E6FF56EC3AF0E552E552E5522CA88E
:101D80000FD09D0E496E710E4A6E4B6A49C0E6FF38
:101D9000E66E4BC0E6FF56EC3AF0E552E552E552EE
:101DA0002CAC0FD07C0E496E710E4A6E4B6A49C046
:101DB000E6FFE66E4BC0E6FF56EC3AF0E552E55220
:101DC000E5522CAE0FD0630E496E710E4A6E4B6A0F
:101DD00049C0E6FFE66E4BC0E6FF56EC3AF0E5522E
:101DE000E552E5522C6A3FD8050EE15C02E2E16A59
:101DF000E552E16EE552E7CFD9FF1200D9CFE6FFF9
:101E0000E1CFD9FFE652F5C5DFFFDF2A400E496E6C
:101E1000DF50495C01E1DF6A0501F651DF5C01E159
:101E200022D80501F551EA6A000FE96E020EEA2296
:101E3000FE0EDBCFEFFFF52B400EF55D01E1F56BFC
:101E4000F651F55D01E12C84FE0EDBCF49F04A6AC4
:101E500049BE4A6849C0F3FF4AC0F4FFE552E55263
:101E6000E7CFD9FF1200D9CFE6FFE1CFD9FFE65285
:101E70000501F551F65D3DE00501905105E020ECCE
:101E800036F02FEC1EF0F8D70501F651D880F55545
:101E900017E2F651F55DDF6EDFCFE6FFF6514A6AD5
:101EA000000F496E020E4A2249C0E6FF4AC0E6FF13
:101EB00088EC35F0E552E552E552F5C5F6F517D058
:101EC000400ED880F655DF6EDFCFE6FFF6514A6A46
:101ED000000F496E020E4A2249C0E6FF4AC0E6FFE3
:101EE00088EC35F0E552E552E5520501F66B20EC41
:101EF00036F0E552E552E7CFD9FF1200D9CFE6FF21
:101F0000E1CFD9FF040EE126DE6ADD6A020EDB6A4C
:101F1000030EDB6A0501F851EA6A000FE96E030E51
:101F2000EA22EF50E66EE66AAFEC3BF0E552E5528E
:101F3000020EF3CFDBFF0501F82BF851496E4A6A18
:101F4000000E491804E1010E4A1801E1F86B020E77
:101F5000DB50DE6EDD6AF851EA6A000FE96E030EAF
:101F6000EA22EF502C0836E0F851EA6A000FE96ED9
:101F7000030EEA22EF500D082DE0F851EA6A000F37
:101F8000E96E030EEA22EF50E66EE66AAFEC3BF034
:101F9000E552E552030EF3CFDBFF0501F82BF851B4
:101FA000496E4A6A000E491804E1010E4A1801E11F
:101FB000F86B020EDBCF4BF04BC04CF04B6A030EBC
:101FC000DB5000014B24496E000E4C204A6E49C084
:101FD000DEFFDD6E000EDFCF3DF0010EDBCF3EF009
:101FE0004D0E3D1802E1510E3E1801E1D2D14D0EC9
:101FF0003D1802E1520E3E1801E1C8D1320E3D18E3
:1020000002E1530E3E1801E1BED1450E3D1802E13A
:10201000530E3E1801E1B4D1430E3D1802E1510EBA
:102020003E1801E1AAD14B0E3D1802E1430E3E18C5
:1020300001E1A0D14C0E3D1802E1420E3E1801E133
:1020400096D1440E3D1802E14E0E3E1801E18CD1AE
:10205000490E3D1802E14E0E3E1801E182D1420EBA
:102060003D1802E1510E3E1801E178D14C0E3D18A9
:1020700002E1510E3E1801E16ED14C0E3D1802E115
:10208000530E3E1801E164D14E0E3D1802E1510E8F
:102090003E1801E15AD14E0E3D1802E1530E3E1892
:1020A00001E150D1430E3D1802E1530E3E1801E10B
:1020B00046D14D0E3D1802E1450E3E1801E13CD1DE
:1020C000500E3D1802E1510E3E1801E132D1500E82
:1020D0003D1802E1540E3E1801E128D1500E3D1882
:1020E00002E1530E3E1801E11ED14D0E3D1802E1F2
:1020F000530E3E1801E114D1470E3D1802E1500E77
:102100003E1801E10AD1430E3D1802E1500E3E187F
:1021100001E100D1490E3D1802E1430E3E1801E1F4
:10212000F6D0490E3D1802E1520E3E1801E1ECD006
:10213000490E3D1802E1530E3E1801E1E2D0530E64
:102140003D1802E1430E3E1801E1D8D0530E3D1870
:1021500002E1520E3E1801E1CED0530E3D1802E1CD
:10216000530E3E1801E1C4D0530E3D1802E1420E59
:102170003E1801E1BAD0430E3D1802E1420E3E186E
:1021800001E1B0D0430E3D1802E1520E3E1801E1CC
:10219000A6D04F0E3D1802E1420E3E1801E19CD040
:1021A000570E3D1802E14D0E3E1801E193D0520E3C
:1021B0003D1802E14D0E3E1801E18AD0440E3D1853
:1021C00002E1500E3E1801E181D04F0E3D1802E1B0
:1021D000500E3E1801E177D0490E3D1802E1500E35
:1021E0003E186EE0580E3D1802E1540E3E1865E0B0
:1021F000540E3D1801E13E505EE0410E3D1801E1F4
:102200003E5057E0560E3D1801E13E5050E0490E59
:102210003D1801E13E5049E04F0E3D1801E13E50AE
:1022200042E0550E3D1802E1430E3E183AE0580ECA
:102230003D1802E1430E3E1831E0430E3D1801E126
:102240003E502AE0520E3D1801E13E5023E0580E68
:102250003D1802E1520E3E181AE0030EDB5001E079
:102260009BD0020EDBCFE6FFE66ADBCFE6FFE66A35
:10227000400E496E710E4A6E4B6A49C0E6FFE66E2B
:102280004BC0E6FF56EC3AF04C6E070EA3D076EC4E
:1022900017F0A2D0D7D8A0D06CD99ED078EC17F088
:1022A0009BD0D4D899D023DA97D0AADA95D0C8DABF
:1022B00093D0D6DA91D012D98FD074EC17F08CD09D
:1022C000F3EC15F089D090EC16F086D0A6DB84D024
:1022D00062DB82D022DB80D02CEC18F07DD07AEC4F
:1022E00017F07AD02AEC18F077D02EEC18F074D0D2
:1022F00030EC18F071D032EC18F06ED034EC18F0ED
:102300006BD036EC18F068D038EC18F065D03AECA9
:1023100018F062D03CEC18F05FD0CDEC18F05CD037
:10232000F7EC29F059D0E9EC2BF056D0B1EC2BF0BA
:1023300053D096EC2BF050D07FEC2CF04DD0AFEC7E
:1023400028F04AD028EC2DF047D058EC2DF044D09E
:1023500072EC2DF041D084EC2DF03ED09FEC2DF0AE
:102360003BD00AEC2DF038D01BEC2DF035D00AEC28
:1023700019F032D012EC19F02FD0BCEC2DF02CD08B
:1023800021EC2EF029D037EC37F026D094EC2EF04B
:1023900023D095EC2EF020D0030EDBCFE6FFE66ACB
:1023A000020EDBCFE6FFE66A030EDBCFE6FFE66A4E
:1023B000020EDBCFE6FFE66A180E496E710E4A6E1A
:1023C0004B6A49C0E6FFE66E4BC0E6FF56EC3AF0BA
:1023D0004C6E0B0EE15E4C500501F851EA6A000F9D
:1023E000E96E030EEA22EF500D080DE02C500BE1D0
:1023F000520E496E4A6ADF50491803E1DE52DD5041
:102400004A1801E02C8EF7C5F8F5040EE15C02E2F3
:10241000E16AE552E16EE552E7CFD9FF120005010E
:10242000FD510FE0F20E496E770E4A6E4B6A49C0BD
:10243000E6FFE66E4BC0E6FF56EC3AF0E552E55299
:10244000E55212004AEC0CF00FEF12F0D9CFE6FF84
:10245000E1CFD9FF030EE126E66AD9CFE6FFDACF56
:10246000E6FF010EE66E4CEC1AF0E552E552E5523D
:10247000E552E66AD950010FE66E000EDA20E66EEC
:10248000020EE66E4CEC1AF0E552E552E552E552CA
:102490002C501AE1DF0417E1D950010FE96EDACFB1
:1024A000EAFFEE50ED100AE0010E496E4A6ADB5079
:1024B000491808E1020EDB504A1804E1010EDBCF97
:1024C000FDF501D02C8CABDF030EE15C02E2E16A8A
:1024D000E552E16EE552E7CFD9FF1200D9CFE6FF12
:1024E000E1CFD9FF030EE126020EDB6AE66A1F0E7A
:1024F000E66E000EE66E030EE66E4CEC1AF0E55248
:10250000E552E552E552E66AD950020FE66E000E3A
:10251000DA20E66E010EE66E4CEC1AF0E552E5525A
:10252000E552E5522C501BE1020EDB500CE11F502E
:10253000201003E1216A226A11D076841FC021F0A5
:1025400020C022F00BD01F50201003E1266A276A1A
:1025500005D076841FC026F020C027F060DF030E70
:10256000E15C02E2E16AE552E16EE552E7CFD9FFB4
:102570001200D9CFE6FFE1CFD9FF0A0EE126E66AC5
:10258000D9CFE6FFDACFE6FF010EE66E4CEC1AF08B
:10259000E552E552E552E552E66AD950010FE66E82
:1025A000000EDA20E66E010EE66E4CEC1AF0E552F3
:1025B000E552E552E552E66AD950020FE66E000E8A
:1025C000DA20E66E010EE66E4CEC1AF0E552E552AA
:1025D000E552E552E66AD950040FE66E000EDA20A5
:1025E000E66E010EE66E4CEC1AF0E552E552E5524D
:1025F000E552E66AD950050FE66E000EDA20E66E67
:10260000010EE66E4CEC1AF0E552E552E552E55249
:10261000E66AD950060FE66E000EDA20E66E010E6D
:10262000E66E4CEC1AF0E552E552E552E552E66AE8
:10263000D950070FE66E000EDA20E66E010EE66E48
:102640004CEC1AF0E552E552E552E552E66AD950F3
:10265000080FE66E000EDA20E66E010EE66E4CEC18
:102660001AF0E552E552E552E552E66AD950090FF3
:10267000E66E000EDA20E66E010EE66E4CEC1AF005
:10268000E552E552E552E552E66AD950030FE66E8F
:10269000000EDA20E66E010EE66E4CEC1AF0E55202
:1026A000E552E552E5522C5018E1DF50926E010ED2
:1026B000DB50936E020EDB50946E040EDB50956E71
:1026C000050EDB50966E030EDB500C0805E20C0E77
:1026D000F36E030EF3CFDBFFA2DE0A0EE15C02E233
:1026E000E16AE552E16EE552E7CFD9FF1200D9CF9A
:1026F000E6FFE1CFD9FF020EE126E66AD9CFE6FF79
:10270000DACFE6FF010EE66E4CEC1AF0E552E55228
:10271000E552E552E76E010EE7CFDBFF2C5066E194
:10272000010EDB5002E1DF50896E010EE66ED9CF5B
:10273000E6FFDACFE6FFE66E4CEC1AF0E552E55222
:10274000E552E552E76E010EE7CFDBFF2C504EE17C
:10275000010EDB5002E1DF508A6E010EE66ED9CF2A
:10276000E6FFDACFE6FFE66E4CEC1AF0E552E552F2
:10277000E552E552E76E010EE7CFDBFF2C5036E164
:10278000010EDB5002E1DF508B6E010EE66ED9CFF9
:10279000E6FFDACFE6FFE66E4CEC1AF0E552E552C2
:1027A000E552E552E76E010EE7CFDBFF2C501EE14C
:1027B000010EDB5002E1DF508C6E010EE66ED9CFC8
:1027C000E6FFDACFE6FFE66E4CEC1AF0E552E55292
:1027D000E552E552E76E010EE7CFDBFF2C5006E134
:1027E000010EDB5002E1DF508D6E19DE020EE15C5E
:1027F00002E2E16AE552E16EE552E7CFD9FF12004D
:102800008450E66EE66A8350E66EE66A8250E66EB3
:10281000E66A8150E66EE66A8050E66EE66AFB0E76
:10282000496E700E4A6E4B6A49C0E6FFE66E4BC0B9
:10283000E6FF56EC3AF04C6E0D0EE15E4C50120085
:10284000FA0E496E770E4A6E4B6A49C0E6FFE66E95
:102850004BC0E6FF56EC3AF0E552E552E552120065
:10286000D9CFE6FFE1CFD9FFE652DF6AF90E496E14
:10287000700E4A6E4B6A49C0E6FFE66E4BC0E6FF3B
:1028800056EC3AF0E552E552E552DF6A2B50DF5C38
:1028900030E2DFCF49F04A6A49BE4A68060E4A0272
:1028A000F3CF4AF04902F3CF49F0F4504A26000E24
:1028B0004926010E4A222950020D4950F324E96E9F
:1028C0004A50F420EA6EEECFE6FFEFCFE6FFF30EBC
:1028D0004B6E700E4C6E4D6A4BC0E6FFE66E4DC0FF
:1028E000E6FF56EC3AF04E6E050EE15E4E50DF2AE2
:1028F000CDD7F70E496E770E4A6E4B6A49C0E6FF98
:10290000E66E4BC0E6FF56EC3AF0E552E552E55272
:10291000E552E552E7CFD9FF1200D9CFE6FFE1CF6C
:10292000D9FF030EE126E66AD9CFE6FFDACFE6FF4C
:10293000E66E4CEC1AF0E552E552E552E552E66AD5
:10294000D950020FE66E000EDA20E66E010EE66E3A
:102950004CEC1AF0E552E552E552E5522C5011E1EB
:10296000DECF49F0DDCF4AF0000E495C100E4A5828
:1029700007E2DECFE9FFDDCFEAFF020EDBCFEFFF9C
:102980004EDD030EE15C02E2E16AE552E16EE552E2
:10299000E7CFD9FF1200D9CFE6FFE1CFD9FF030E71
:1029A000E126E66AD9CFE6FFDACFE6FFE66E4CEC29
:1029B0001AF0E552E552E552E5522C5024E1DECF03
:1029C00049F0DDCF4AF0000E495C100E4A5807E28C
:1029D000DECFE9FFDDCFEAFF020EEFCFDBFF020E15
:1029E000DBCFE6FFE66AE90E496E700E4A6E4B6A6F
:1029F00049C0E6FFE66E4BC0E6FF56EC3AF04C6E7F
:102A0000050EE15E4C50030EE15C02E2E16AE55224
:102A1000E16EE552E7CFD9FF1200D9CFE6FFE1CF53
:102A2000D9FF030EE126E66AD9CFE6FFDACFE6FF4B
:102A3000050EE66E4CEC1AF0E552E552E552E55211
:102A4000E66AD950010FE66E000EDA20E66E010E3E
:102A5000E66E4CEC1AF0E552E552E552E552E66AB4
:102A6000D950020FE66E000EDA20E66E010EE66E19
:102A70004CEC1AF0E552E552E552E5522C5001E0DB
:102A8000A8D0020EDB50010801E2A0D0010EDB50FD
:102A9000070801E29BD0410E496EDF50495C1AE104
:102AA000020EDB500CE1010EF36EDB5004E0D89017
:102AB000F336E806FCE1F350F31C921689D0010EC0
:102AC000F36EDB5004E0D890F336E806FCE1F350F7
:102AD00092127ED0420E496EDF50495C1AE1020E1E
:102AE000DB500CE1010EF36EDB5004E0D890F336BE
:102AF000E806FCE1F350F31C93166AD0010EF36E66
:102B0000DB5004E0D890F336E806FCE1F350931272
:102B10005FD0430E496EDF50495C1AE1020EDB5074
:102B20000CE1010EF36EDB5004E0D890F336E806BA
:102B3000FCE1F350F31C94164BD0010EF36EDB5006
:102B400004E0D890F336E806FCE1F350941240D04C
:102B5000440E496EDF50495C1AE1020EDB500CE175
:102B6000010EF36EDB5004E0D890F336E806FCE18A
:102B7000F350F31C95162CD0010EF36EDB5004E0DD
:102B8000D890F336E806FCE1F350951221D0450EBB
:102B9000496EDF50495C1AE1020EDB500CE1010E78
:102BA000F36EDB5004E0D890F336E806FCE1F35016
:102BB000F31C96160DD0010EF36EDB5004E0D89096
:102BC000F336E806FCE1F350961202D02C8C01D0CB
:102BD00026DC030EE15C02E2E16AE552E16EE552B9
:102BE000E7CFD9FF1200D9CFE6FFE1CFD9FF030E1F
:102BF000E126020EDB6AE66AD9CFE6FFDACFE6FF0E
:102C0000050EE66E4CEC1AF0E552E552E552E5523F
:102C1000E66AD950010FE66E000EDA20E66E010E6C
:102C2000E66E4CEC1AF0E552E552E552E5522C50B6
:102C30006DE1010EDB50070854E3410E496EDF5091
:102C4000495C0BE1010EF36EDB5004E0D890F336E3
:102C5000E806FCE1F35080143FD0420E496EDF508D
:102C6000495C0BE1010EF36EDB5004E0D890F336C3
:102C7000E806FCE1F35081142FD0430E496EDF507B
:102C8000495C0BE1010EF36EDB5004E0D890F336A3
:102C9000E806FCE1F35082141FD0440E496EDF5069
:102CA000495C0BE1010EF36EDB5004E0D890F33683
:102CB000E806FCE1F35083140FD0450E496EDF5057
:102CC000495C0FE1010EF36EDB5004E0D890F3365F
:102CD000E806FCE1F3508414E76E020EE7CFDBFF59
:102CE00002D02C8C13D0DBCFE6FFE66AE00E496EF3
:102CF000700E4A6E4B6A49C0E6FFE66E4BC0E6FFB7
:102D000056EC3AF04C6E050EE15E4C50030EE15C61
:102D100002E2E16AE552E16EE552E7CFD9FF120027
:102D2000D9CFE6FFE1CFD9FF030EE126E66AD9CF7E
:102D3000E6FFDACFE6FF050EE66EAEDBE552E552C2
:102D4000E552E552E66AD950010FE66E000EDA2030
:102D5000E66E010EE66EA0DBE552E552E552E55265
:102D6000E66AD950020FE66E000EDA20E66E010E1A
:102D7000E66E92DBE552E552E552E5522C5001E059
:102D8000A9D0020EDB50010801E2A0D0010EDB50F9
:102D9000070801E29BD0410E496EDF50495C1AE101
:102DA000020EDB500CE1010EF36EDB5004E0D89014
:102DB000F336E806FCE1F350F31C891689D0010EC6
:102DC000F36EDB5004E0D890F336E806FCE1F350F4
:102DD00089127ED0420E496EDF50495C1AE1020E24
:102DE000DB500CE1010EF36EDB5004E0D890F336BB
:102DF000E806FCE1F350F31C8A166AD0010EF36E6C
:102E0000DB5004E0D890F336E806FCE1F3508A1278
:102E10005FD0430E496EDF50495C1AE1020EDB5071
:102E20000CE1010EF36EDB5004E0D890F336E806B7
:102E3000FCE1F350F31C8B164BD0010EF36EDB500C
:102E400004E0D890F336E806FCE1F3508B1240D052
:102E5000440E496EDF50495C1AE1020EDB500CE172
:102E6000010EF36EDB5004E0D890F336E806FCE187
:102E7000F350F31C8C162CD0010EF36EDB5004E0E3
:102E8000D890F336E806FCE1F3508C1221D0450EC1
:102E9000496EDF50495C1AE1020EDB500CE1010E75
:102EA000F36EDB5004E0D890F336E806FCE1F35013
:102EB000F31C8D160DD0010EF36EDB5004E0D8909C
:102EC000F336E806FCE1F3508D1202D02C8C02D0D0
:102ED0000FEC12F0030EE15C02E2E16AE552E16EF2
:102EE000E552E7CFD9FF12000FEF12F00FEF12F00B
:102EF0000FEF12F0D9CFE6FFE1CFD9FF040EE126A4
:102F0000E66AD9CFE6FFDACFE6FF050EE66EC4DA51
:102F1000E552E552E552E552E66AD950010FE66EF8
:102F2000000EDA20E66E010EE66EB6DAE552E552E4
:102F3000E552E552E66AD950020FE66E000EDA203D
:102F4000E66E030EE66EA8DAE552E552E552E5526A
:102F50002C5076E1D950020FE96EDACFEAFF720EFB
:102F6000D880EE542E0EED5441E3D950020FE96E95
:102F7000DACFEAFFEE50ED101FE04C684D684E6A64
:102F80002D0EE76E020EDBCF4FF0030EDBCF50F0BD
:102F9000E7504F26000E5022516A4F504C5C496E4C
:102FA00050504D584A6E51504E584B6E020E49C00B
:102FB000DBFF030E4AC0DBFF010EDB50070816E300
:102FC000410E496EDF50495C02E1DF6A11D0420ECA
:102FD000496EDF50495C02E1080E06D0430E496E8F
:102FE000DF50495C03E1100EDF6E02D02C8C28D03C
:102FF000010EDB50DF24E96EEA6AD890E936EA3642
:10300000690EE926010EEA22020EDBCFEEFF030E67
:10301000DBCFEDFF010EDB50DF24EA6A510FE96ED2
:10302000010EEA22EF040AE1010EDB50DF24EA6A16
:10303000510FE96E010EEA22020EEF6E0FEC12F054
:10304000040EE15C02E2E16AE552E16EE552E7CF8F
:10305000D9FF12000FEF12F00FEF12F00FEF12F086
:103060000FEF12F00FEF12F00FEF12F00FEF12F060
:103070000FEF12F00FEF12F0D9CFE6FFE1CFD9FF3B
:10308000070EE126E66AD9CFE6FFDACFE6FF030EA8
:10309000E66E02DAE552E552E552E552E66AD950AB
:1030A000020FE66E000EDA20E66E030EE66EF4D92D
:1030B000E552E552E552E5522C5065E1DECF9AF13A
:1030C000DDCF9BF1020EDBCFA2F1030EDBCFA3F12C
:1030D000040EDB6A030EF36E040EDBCFF4FFF35035
:1030E000F45C4FE2010EE66ED9CFE6FFDACFE6FFE1
:1030F000030EE66ED1D9E552E552E552E552E76E90
:10310000050EE7CFDBFF010EE66ED950020FE66E2B
:10311000000EDA20E66E030EE66EBED9E552E552E9
:10312000E552E552E76E060EE7CFDBFF2C502BE1B0
:10313000050EDB5026E1060EDB5023E1040EDB28F2
:10314000E96EEA6AD890E936EA369A0EE926010E67
:10315000EA22DECFEEFFDDCFEDFF040EDB28E96EC5
:10316000EA6AD890E936EA36A20EE926010EEA228A
:10317000020EDBCFEEFF030EDBCFEDFF040EDB2AEA
:10318000A9D70FEC12F0070EE15C02E2E16AE5520A
:10319000E16EE552E7CFD9FF1200D9CFE6FFE1CFCC
:1031A000D9FFE652E66AD9CFE6FFDACFE6FF010E95
:1031B000E66E72D9E552E552E552E5522C500DE12A
:1031C000DF5007E0F00E9314936E0101010E996F2A
:1031D00002D00101996B0FEC12F0E552E552E7CFF6
:1031E000D9FF1200D9CFE6FFE1CFD9FFE652DF6A5F
:1031F000FF0EDF5C0AE2E868E85005E0E80600D070
:1032000000D000D0F9D7DF2AF3D7E552E552E7CF57
:10321000D9FF1200F29EF29C6592656AE3DF0FEF20
:1032200000F01200D9CFE6FFE1CFD9FF100EE12662
:10323000E66AD950010FE66E000EDA20E66EE66A05
:103240002BD9E552E552E552E552E66AD9CFE6FFC1
:10325000DACFE6FF010EE66E1FD9E552E552E552E0
:10326000E552E66AD950040FE66E000EDA20E66EEB
:10327000020EE66E11D9E552E552E552E552E66AD4
:10328000D950020FE66E000EDA20E66E030EE66EEF
:1032900003D9E552E552E552E552E66AD9500A0FE4
:1032A000E66E000EDA20E66E060EE66EF5D8E55202
:1032B000E552E552E552E66AD950060FE66E000E79
:1032C000DA20E66E070EE66EE7D8E552E552E552E3
:1032D000E552E66AD9500E0FE66E000EDA20E66E71
:1032E000040EE66ED9D8E552E552E552E552E66A9B
:1032F000D9500F0FE66E000EDA20E66E050EE66E70
:10330000CBD8E552E552E552E552010EDBCF49F04C
:103310004A6A49BE4A6849C0E6FF4AC0E6FFD40E81
:103320004B6E700E4C6E4D6A4BC0E6FFE66E4DC0A4
:10333000E6FF56EC3AF04E6E050EE15E4E50DFCFE2
:10334000E6FFE66AC80E496E700E4A6E4B6A49C0C7
:10335000E6FFE66E4BC0E6FF56EC3AF04C6E050E0B
:10336000E15E4C50040EDBCFE6FF050EDBCFE6FF3F
:10337000BC0E496E700E4A6E4B6A49C0E6FFE66E9F
:103380004BC0E6FF56EC3AF04C6E050EE15E4C5039
:10339000020EDBCFE6FF030EDBCFE6FFB00E496E79
:1033A000700E4A6E4B6A49C0E6FFE66E4BC0E6FF00
:1033B00056EC3AF04C6E050EE15E4C50D9500A0FB7
:1033C000E96EDACFEAFFEECFE6FFEECFE6FFEECF13
:1033D000E6FFEFCFE6FFA30E496E700E4A6E4B6A12
:1033E00049C0E6FFE66E4BC0E6FF56EC3AF04C6E85
:1033F000070EE15E4C50D950060FE96EDACFEAFFB6
:10340000EECFE6FFEECFE6FFEECFE6FFEFCFE6FF33
:10341000960E496E700E4A6E4B6A49C0E6FFE66E24
:103420004BC0E6FF56EC3AF04C6E070EE15E4C5096
:103430000E0EDBCFE6FFE66A8A0E496E700E4A6E0C
:103440004B6A49C0E6FFE66E4BC0E6FF56EC3AF029
:103450004C6E050EE15E4C500F0EDBCFE6FFE66AC8
:103460007E0E496E700E4A6E4B6A49C0E6FFE66EEC
:103470004BC0E6FF56EC3AF04C6E050EE15E4C5048
:103480000FEC12F0100EE15C02E2E16AE552E16E2F
:10349000E552E7CFD9FF1200D9CFE6FFE1CFD9FF40
:1034A000090EE126080EDB6A0D0E496E0501F85182
:1034B000EA6A000FE96E030EEA22EF50495C05E16B
:1034C000FB0EDB5044E12C8842D0F851EA6A000F31
:1034D000E96E030EEA22EF502C081FE0FB0EDB50D2
:1034E0001AE1F851EA6A000FE96E030EEA22EF5082
:1034F000E66EE66A570E496E700E4A6E4B6A49C018
:10350000E6FFE66E4BC0E6FF56EC3AF04C6E050E59
:10351000E15E4C502C8A020EE5D1F82BF851496E31
:103520004A6A000E491804E1010E4A1801E1F86BDD
:103530000D0E496EF851EA6A000FE96E030EEA2299
:10354000EF50495C06E1FB0EDB5001E12C88030ED5
:10355000C9D12D0E496EF851EA6A000FE96E030ECB
:10356000EA22EF50495C2EE1040E4A6EFE0EDB505B
:103570004A5C28E0050E4B6EFE0EDB504B5C22E0F1
:10358000FE0EDB0401E147D1030E496EFE0EDB5057
:10359000495C01E140D1070E4A6EFE0EDB504A5CE9
:1035A00001E139D1010EF36E080EF3CFDBFFF82BEA
:1035B000F851496E4A6A000E491804E1010E4A1892
:1035C00001E1F86B040E496EFE0EDB50495C11E020
:1035D000050E4A6EFE0EDB504A5C0BE00A0EE66EEC
:1035E000D9CFE6FFDACFE6FF89D9E552E552E552B9
:1035F00042D0F851EA6A000FE96E030EEA22EFCFDB
:1036000049F0000E49C0DFFF010EDB6A020EDB6AE3
:10361000030EDB6A050E496EFE0EDB50495C1FE1AE
:10362000000EDFCFE6FF010EDBCFE6FFAFEC3BF095
:10363000E552E552F3CF49F0F4CF4AF04B6A4C6AB9
:103640004AAE02D04B684C6849C0DFFF010E4AC049
:10365000DBFF020E4BC0DBFF030E4CC0DBFF05019E
:10366000F82BF851496E4A6A000E491804E1010E20
:103670004A1801E1F86B080EDB506FE0FE0EDB50DC
:103680000FE1D9CFE9FFDACFEAFFD880800EEE5400
:10369000000EEE54000EEE54000EEE5401E2BBD0CC
:1036A000020E496EFE0EDB50495C0FE1D9CFE9FFF7
:1036B000DACFEAFFD880000EEE54800EEE54000EF2
:1036C000EE54000EEE5401E2A6D0060E4A6EFE0E37
:1036D000DB504A5C0FE1D9CFE9FFDACFEAFFD880AF
:1036E000000EEE54000EEE54000EEE54800EEE541A
:1036F00001E291D0D9CFE9FFDACFEAFF040EEECF95
:10370000DBFF050EEECFDBFF060EEECFDBFF070E75
:10371000EECFDBFF080EDB5001E196D0040EDBCFCD
:103720003BF0050EDBCF3CF0060EDBCF3DF0070E85
:10373000DBCF3EF0406841684268436877EC3BF07D
:10374000040E37C0DBFF050E38C0DBFF060E39C0A4
:10375000DBFF070E3AC0DBFF77D0FE0EDB500EE139
:10376000D9CFE9FFDACFEAFFD8807F0EEE54000E02
:10377000EE54000EEE54000EEE544DE3FE0EDB044C
:103780000EE1D9CFE9FFDACFEAFFD880FF0EEE5481
:10379000000EEE54000EEE54000EEE543CE3020E0A
:1037A000496EFE0EDB50495C0EE1D9CFE9FFDACF5E
:1037B000EAFFD880FF0EEE547F0EEE54000EEE545A
:1037C000000EEE5428E3030E4A6EFE0EDB504A5CF8
:1037D0000EE1D9CFE9FFDACFEAFFD880FF0EEE5431
:1037E000FF0EEE54000EEE54000EEE5414E3060EDF
:1037F0004B6EFE0EDB504B5C11E1D9CFE9FFDACF07
:10380000EAFFD880FF0EEE54FF0EEE54FF0EEE548A
:103810007F0EEE5403E22C8C010E64D0070E496E2D
:10382000FE0EDB50495C10E0D9CFE9FFDACFEAFFAA
:10383000040EEECFDBFF050EEECFDBFF060EEECF64
:10384000DBFF070EEECFDBFFFE0EDB50070A38E092
:10385000010A25E0050A16E0010A14E0030A08E05F
:10386000050A06E0010A04E0050A02E0040E3AD067
:10387000FC0EDBCFE9FFFD0EDBCFEAFF040EDBCF52
:10388000EFFF2FD0FC0EDBCFE9FFFD0EDBCFEAFF11
:10389000040EDBCFEEFF050EDBCFEDFF22D0FC0EDA
:1038A000DBCFE9FFFD0EDBCFEAFF040EDBCFEEFF3F
:1038B000050EDBCFEEFF060EDBCFEEFF070E0FD0BF
:1038C000FC0EDBCFE9FFFD0EDBCFEAFFDFCFEEFF23
:1038D000010EDBCFEEFF020EDBCFEEFF030EDBCFE0
:1038E000EEFF000E496E090EE15C02E2E16AE5526C
:1038F000E16E4950E552E7CFD9FF1200D9CFE6FF7C
:10390000E1CFD9FF020EE126FD0EDBCFE9FFFE0E6F
:10391000DBCFEAFFEE6AEE6AEE6AEE6A010EDB6A60
:10392000FC0EDB50F36E010EDBCFF4FFF350F45CC2
:1039300062E20501F851EA6A000FE96E030EEA221D
:10394000EFCFDFFF300EDF5C51E3DF5039084EE38D
:10395000FD0EDBCFE9FFFE0EDBCFEAFFEECF49F035
:10396000EECF4AF0EECF4BF0EFCF4CF00A0E406EA8
:10397000416A426A436A49C03BF04AC03CF04BC0CE
:103980003DF04CC03EF077EC3BF037C049F038C01A
:103990004AF039C04BF03AC04CF0300EDF5C4D6E4F
:1039A0004E6A4F6A506AE85049264E504A224F509C
:1039B0004B2250504C22FD0EDBCFE9FFFE0EDBCF39
:1039C000EAFF49C0EEFF4AC0EEFF4BC0EEFF4CC01D
:1039D000EEFF0501F82BF851496E4A6A000E4918AE
:1039E00007E1010E4A1804E1F86B02D0000E04D082
:1039F000010EDB2A95D7010E496E020EE15C02E250
:103A0000E16AE552E16E4950E552E7CFD9FF120075
:103A10002550E66EE66A4B0E496E700E4A6E4B6A92
:103A200049C0E6FFE66E4BC0E6FF56EC3AF04C6E3E
:103A3000050EE15E4C5012000501A85108E0010E90
:103A4000496E6550020B01E0010E495C1BE101016A
:103A5000FA07000EFB5BFC510BE1FA51FB1111E17F
:103A60008C86A00EFA6F0F0EFB6F010EFC6F12001A
:103A7000FA51FB1163E18C96A00EFA6F0F0EFB6FEB
:103A8000FC6B1200A80509E0020EA85D06E0040E1A
:103A9000A85D03E0100EA85D1BE10101FA07000E0E
:103AA000FB5BFC510BE1FA51FB1111E18C86200EFE
:103AB000FA6F4E0EFB6F010EFC6F1200FA51FB11F4
:103AC0003DE18C96200EFA6F4E0EFB6FFC6B1200E0
:103AD000200EA85D33E10101FA07000EFB5BFC51EB
:103AE0000AE1FA51FB112AE18C86100EFA6F270EBB
:103AF000FB6F010E18D0FC050AE1FA51FB111EE123
:103B00008C96100EFA6F270EFB6F020E0CD0020E71
:103B1000FC5D0BE1FA51FB1111E18C86A00EFA6FEE
:103B2000860EFB6F030EFC6F1200FA51FB1106E1CB
:0E3B30008C96100EFA6F270EFB6FFC6B1200C6
:023B3E00D9CFDD
:103B4000E6FFE1CFD9FFE652A098636A626A0F01EF
:103B5000266B020EE66EE66AE66A270EE66E0F0E2A
:103B6000E66E09EC3AF0496E050EE15E49500F0130
:103B7000160E396F9F0E376F7B0E366FDF6ADF5080
:103B8000496E4A6A0C0E495C000E4A5810E2DF503A
:103B9000040DF3CFE9FFF4CFEAFF000EE926040E8F
:103BA000EA22EE6AEE6AEE6AEE6ADF2AE8D7658CF0
:103BB0000F01386B6598659C62A607D06296050177
:103BC000BF6BC46BC56BC66BF7D70501010ED86F11
:103BD000D96FDA6BDB6BCC6BDF6A030EDF5C26E23E
:103BE000EA6ADF34FE0BEA36E96EB50EE926050E09
:103BF000EA22EE6AED6AEA6ADF34FE0BEA36E96E23
:103C0000AF0EE926050EEA22EE6AED6ADF50EA6A97
:103C1000D00FE96E050EEA22EF6ADF50EA6AD30F91
:103C2000E96E050EEA22EF6ADF2AD7D70501080EF2
:103C3000B56F040EB66F0F01160E266F0401300E1D
:103C4000026F040E036F400E016F840E006F0501BA
:103C5000A96BA86BE552E552E7CFD9FF1200D9CF87
:103C6000E6FFE1CFD9FFE6520501A85110E1656AF0
:103C70000F01366B160E396F9F0E376F7B0E366F46
:103C800065B602D06586FCD70501010EA86FA805B0
:103C90000AE165BA08D0626A0F01366B368136894F
:103CA0000501020EA86F6250040B06E00F013651A9
:103CB000040B02E06294CDD865B25BD06250010B78
:103CC00009E00F013651010B05E039DF0501040E53
:103CD000A86F62906250100B06E00F013651100B76
:103CE00002E0A1D8629862AC1AD00F0136AD0FD0B5
:103CF000010EE66EE66A000EE66EE66A730EE66E8A
:103D0000E66A70EC39F0496E060EE15E4950629C3D
:103D10000501D65101E0D607D65101E151DB6250D1
:103D2000200B05E00F013651200B01E062D86250F4
:103D3000020B14E00F013651020B10E0010EE66E8B
:103D4000E66A000EE66EE66AE6687F0EE66E70ECE6
:103D500039F0496E060EE15E4950636A040E0501B2
:103D6000E76EA819E8AE02D0E73402D0E750A85DAC
:103D700002E2A19839D00F0136A735D0DF6A040ED0
:103D8000DF5C31E262A62FD064CFCDF50501CD51C5
:103D9000780BE842E842E842CE6F6296CDB506D095
:103DA000CE51EA6AD30FE96E050E05D0CE51EA6A0C
:103DB000D00FE96E050EEA22EF70CE5102E161D814
:103DC00010D0000EE66EE66ACD0EE66E050EE66ECB
:103DD000720EE66EE66A70EC39F0496E060EE15E30
:103DE0004950DF2ACCD7A198E552E552E7CFD9FF59
:103DF00012000F0126A115D0ABC5E9FFACC5EAFF43
:103E0000EF5080080DE1B5C5E9FFB6C5EAFFEF50F8
:103E1000840806E1ABC5E9FFACC5EAFF8C0EEF6E86
:103E20002691629A12000F0136856298658205011B
:103E3000010ECC6F000EE66EE66AE66EE66A750E5F
:103E4000E66EE66A70EC39F0496E060EE15E4950A6
:103E500012000501CC6B000EE66EE66AE66EE66ABD
:103E6000740EE66EE66A70EC39F0496E060EE15E9D
:103E7000495065920F01369562A402D06294FCD736
:103E80001200D9CFE6FFE1CFD9FFE65205012D0E92
:103E9000D66FFD0ECD1553E17E0ECD15E8407F0B9C
:103EA000040DF3CFABF5F4CFACF5000EAB27040E49
:103EB000AC23ABC5ADF5ACC5AEF5AD75ABC5E9FF93
:103EC000ACC5EAFFEF503C0BE842E8420D0835E193
:103ED000DF6A080EDF5C23E2ABC5E9FFACC5EAFF91
:103EE000020EE926000EEA22EE50EFCFEAFFE96E5D
:103EF000EF50E66EDF50EA6A300FE96E040EEA22F8
:103F0000E552E750EF6EABC5E9FFACC5EAFF020E24
:103F1000E926000EEA22EE2AEF22DF2ADAD7ABC525
:103F2000E9FFACC5EAFF020EE926000EEA22300ED8
:103F3000EE6E040EED6E0DD807D03AD805D0FD0E0A
:103F4000CD15040801E159D8E552E552E7CFD9FF74
:103F500012000501BB6BD76BDA6BDB6BCF6BBC6BF5
:103F6000B5C5E9FFB6C5EAFFEF9EB575B5C5E9FF72
:103F7000B6C5EAFFEF9EB575ADC5E9FFAEC5EAFF70
:103F8000EF9EBF6BC06BC16BC46BC56BC66B8FD82C
:103F9000000EE66EE66AE66EE66A030EE66EE66A16
:103FA00070EC39F0496E060EE15E495026EF23F0C1
:103FB000020E0501BC5D02E1E6EF23F0BC6BCF51C0
:103FC0001AE1ADC5E9FFAEC5EAFFEE52400EEF6E55
:103FD000ADC5E9FFAEC5EAFF020EE926000EEA22F2
:103FE000300EEE6E040EED6EADC5E9FFAEC5EAFF14
:103FF0008C0EEF6E1200CF6B1200D9CFE6FFE1CF2F
:10400000D9FFE652B5C5E9FFB6C5EAFFEF50400B50
:1040100001E0010EDF6E0501B575080EA85D0BE12C
:1040200032C438FF0F01385103E00501100E02D0F1
:104030000501040EA86FBC0526E1B5C5E9FFB6C5AC
:10404000EAFF020EE926000EEA22380EEE6E040E9A
:10405000ED6E5DDB020E0501BB5D06E1B5C5E9FF56
:10406000B6C5EAFF840E0DD0DF5006E1B5C5E9FF05
:10407000B6C5EAFFC80E05D0B5C5E9FFB6C5EAFF6B
:10408000880EEF6E0FD0C4AF0CD0C751C81107E037
:1040900005D0C8C5FAFF0501C751F96EFADF050161
:1040A000C49FBC6BE552E552E7CFD9FF1200040173
:1040B0003051600BE842E842E842E842E842000939
:1040C00001E0120031510C0A50E00B0A3FE00C0AEB
:1040D00031E0010A22E00B0A1EE0020A1CE0030A9A
:1040E00018E0080A10E0010A0CE00F0A08E0030AD1
:1040F00001E012000501BF8F080EA86F12006FEFDC
:1041000022F085EF24F00501A90EBD6F050EBE6FEC
:104110000CD0CCEF22F0B6EF20F034510501BD6F8A
:10412000BE6BAA0EBD27050EBE23BF81010EC06F58
:10413000BF8F12000501BF8F04013451EA6AAA0F34
:10414000E96E050EEA2232C4EFFF1200000EE66EA1
:10415000E66AE66EE66A020EE66EE66A70EC39F032
:10416000496E060EE15E495012001200D9CFE6FFFB
:10417000E1CFD9FF030EE1260401320510E13051F1
:104180001F0B00090CE10501BF8F030E0401315D17
:1041900004E10501010ECB6F02D00501CB6B0401D8
:1041A000325101E003D130511F0B020801E0FED073
:1041B00034510F0B000901E1F9D034510F0B020803
:1041C00001E2F4D0200E0501A85D01E0EFD0BF8F21
:1041D000040134BF16D034510F0BE96EEA6AD8904F
:1041E000E936EA36AF0EE926050EEA22EECFDEFF0B
:1041F000EDCFDDFF34510F0BEA6AD30FE96E050EE8
:1042000015D034510F0BE96EEA6AD890E936EA36D8
:10421000B50EE926050EEA22EECFDEFFEDCFDDFF7B
:1042200034510F0BEA6AD00FE96E050EEA22020E36
:10423000EFCFDBFFD950020FE96EDACFEAFFEF5084
:10424000010B03E1000EDF9401D0DF8434BF0BD0FB
:1042500034510F0BE96EEA6AD890E936EA36AF0EB0
:10426000E926050E0AD034510F0BE96EEA6AD890A0
:10427000E936EA36B50EE926050EEA22DECFEEFF74
:10428000DDCFEDFF030E315D20E1DECFE9FFDDCFB5
:10429000EAFFEF50800B11E034BF07D034510F0B11
:1042A000EA6AD30FE96E050E06D034510F0BEA6AA5
:1042B000D00FE96E050EEA22EF82840EDECFE9FF11
:1042C000DDCFEAFFE850EF1271D0DF74DECFE9FFF7
:1042D000DDCFEAFFEF50800B1BE0DECFE9FFDDCF43
:1042E000EAFFEF9EDECFE9FFDDCFEAFFEF8C020EA3
:1042F000E66EE66ADECFE6FFDDCFE6FF050EE66E90
:10430000E66A70EC39F0496E060EE15E495005D060
:10431000DECFE9FFDDCFEAFFEF8CDF74D950020F6B
:10432000E96EDACFEAFFEF50020B0EE1DECFE9FFD4
:10433000DDCFEAFFEF50800B32E0DECFE9FFDDCFCB
:10434000EAFFEF50040B2BE1040134BF07D03451D6
:104350000F0BEA6AD30FE96E050E06D034510F0B2E
:10436000EA6AD00FE96E050EEA22EF923B0E496E23
:10437000DECFE9FFDDCFEAFFE850EF16020EE66E72
:10438000E66ADECFE6FFDDCFE6FF050EE66EE66A03
:1043900070EC39F0496E060EE15E495007D03B0ED5
:1043A000DECFE9FFDDCFEAFFE850EF16030EE15C58
:1043B00002E2E16AE552E16EE552E7CFD9FF120071
:1043C0000501D8514DE1010ED86FD95149E1010ED7
:1043D000D96F020EBC5D0DE1B5C5E9FFB6C5EAFFB8
:1043E000EE52EF6AB5C5E9FFB6C5EAFFC80EEF6E3B
:1043F0001200BC0535E1CF6BABC5E9FFACC5EAFFE8
:10440000EE52400EEF6EABC5E9FFACC5EAFF020EFF
:10441000E926000EEA22300EEE6E040EED6EABC5FC
:10442000E9FFACC5EAFF840EEF6E010ECF6FADC59C
:10443000E9FFAEC5EAFFEE52400EEF6EADC5E9FFF3
:10444000AEC5EAFF020EE926000EEA22300EEE6E3D
:10445000040EED6EADC5E9FFAEC5EAFF800EEF6E4E
:1044600012000501DA6BDB6B020EBC5D18E1ADC515
:10447000E9FFAEC5EAFFEE52400EEF6EADC5E9FFB3
:10448000AEC5EAFF020EE926000EEA22380EEE6EF5
:10449000040EED6EADC5E9FFAEC5EAFF1DD0C051FB
:1044A0000401365D0501C1510401375904E236C4E7
:1044B000C0F537C4C1F52BD9B5C5E9FFB6C5EAFFCC
:1044C000020EE926000EEA22380EEE6E040EED6EA4
:1044D000B5C5E9FFB6C5EAFFC80EEF6E1200800E43
:1044E0000401305D58E10501C00EBF6F0401335176
:1044F000030A2FE0010A09E0030A4BE10501DA0E85
:10450000BD6F750EBE6F120E3ED03251F66EF76A59
:10451000D890F636F736610EF626760EF7220900A9
:10452000F5CFBDF50A00F5CFBEF5020E0501F76A1D
:10453000BD25F66EBE51F7220800F5CFC0F5030E7B
:10454000F76ABD25F66EBE51F7220800F5CFC1F51A
:104550001200030E325D1AE23251F66EF76AD890FD
:10456000F636F736630EF626760EF7220900F5CFFB
:10457000BDF50A00F5CFBEF5BDC5F6FFBEC5F7FF18
:104580000800F5500501C06FC16B12000501BF6B3B
:1045900012000501BF6B1200D9CFE6FFE1CFD9FFB2
:1045A000020EE1260401386B396B30511F0B020AF1
:1045B00011E0030A0CE0010A35E10501BF8F040197
:1045C00038810501CB052EE1040138832BD005018C
:1045D000BF8F28D00501BF8F040134BF0BD03451E9
:1045E0000F0BE96EEA6AD890E936EA36AF0EE92693
:1045F000050E0AD034510F0BE96EEA6AD890E936FD
:10460000EA36B50EE926050EEA22EECFDEFFEDCF43
:10461000DDFFDECFE9FFDDCFEAFFEF50040B02E064
:10462000010E386F0501BFAF07D0380EBD6F040E05
:10463000BE6FBF81020EC06F020EE15C02E2E16A52
:10464000E552E16EE552E7CFD9FF1200659805010A
:10465000BFBF2BD0C4AF09D0020EBC6FDB5101E14C
:1046600000DF0501D96BD86B1200ADC5E9FFAEC5FF
:10467000EAFFEE52400EEF6EADC5E9FFAEC5EAFFB0
:10468000020EE926000EEA22300EEE6E040EED6EEA
:10469000ADC5E9FFAEC5EAFF8C0EEF6EB5C5E9FF0B
:1046A000B6C5EAFF840EEF6E1200040130AF0DD0E4
:1046B0000501010EBC6FDA5101E1D3DE0501D96BB2
:1046C000D86BD75123E1E0EF21F00501020EBC6F5A
:1046D000ADC5E9FFAEC5EAFFEE52400EEF6EADC5C7
:1046E000E9FFAEC5EAFF020EE926000EEA22300E0F
:1046F000EE6E040EED6EADC5E9FFAEC5EAFF840EA9
:10470000EF6ED96BD86BD75101E15ADE1200D9CFC9
:10471000E6FFE1CFD9FFE652400EDF6E0501C05D36
:10472000000EC1590AE2C0C5DFFFBB5102E1010E14
:1047300003D0BB0502E1020EBB6FDF504A6AE850AE
:10474000C05DC06F4A50C159C16FB5C5E9FFB6C55C
:10475000EAFFEE52DFCFEFFF380EC96F040ECA6FCB
:10476000BFB118D0DF502DE0BDC5F6FFBEC5F7FFC5
:10477000BD2B000EBE230800F550E66EC9C5E9FF4B
:10478000CAC5EAFFC92B000ECA23E552E750EF6EF7
:10479000DF06E8D7DF5015E0BDC5E9FFBEC5EAFF7B
:1047A000BD2B000EBE23EF50E66EC9C5E9FFCAC59A
:1047B000EAFFC92B000ECA23E552E750EF6EDF0671
:1047C000E9D7E552E552E7CFD9FF1200D9CFE6FF8E
:1047D000E1CFD9FF020EE126ABC5E9FFACC5EAFF88
:1047E000EE52EFCFDFFFDFCF49F049500501C55D45
:1047F000000EC65902E2C5C5DFFFDF50496E4A6AA6
:10480000E850C55DC56F4A50C659C66F010EDB6AD8
:10481000DF50F36E010EDBCFF4FFF350F45C16E2D1
:10482000010EDB50EA6A380FE96E040EEA22EF50FF
:10483000E66EC2C5E9FFC3C5EAFFC22B000EC32363
:10484000E552E750EF6E010EDB2AE2D7000ED8806A
:10485000C555000EC65527E2ADC5E9FFAEC5EAFF56
:10486000EE52400EEF6EADC5E9FFAEC5EAFF020E97
:10487000E926000EEA22380EEE6E040EED6EABC590
:10488000E9FFACC5EAFFEF50400B06E1ADC5E9FF1B
:10489000AEC5EAFFC80E05D0ADC5E9FFAEC5EAFF5B
:1048A000880EEF6E28D0ADC5E9FFAEC5EAFFEE5227
:1048B000400EEF6EADC5E9FFAEC5EAFF020EE92678
:1048C000000EEA22300EEE6E040EED6EADC5E9FF6D
:1048D000AEC5EAFF840EEF6EC751C81107E005D0E0
:1048E000C8C5FAFF0501C751F96EFADF0501C49F7B
:1048F000D75101E165DD020EE15C02E2E16AE552B9
:10490000E16EE552E7CFD9FF1200D9CFE6FFE1CF44
:10491000D9FFE6520501BF8F020EE66EE66AE66A2F
:10492000270EE66E0F0EE66E09EC3AF0496E050EA4
:10493000E15E4950DF6ADF50496E4A6A0C0E495CFD
:10494000000E4A5810E2DF50040DF3CFE9FFF4CF18
:10495000EAFF000EE926040EEA22EE6AEE6AEE6A2B
:10496000EE6ADF2AE8D7658C010EE66EE66AE66A33
:10497000AA0EE66E050EE66E09EC3AF0496E050EDB
:10498000E15E4950659C0501080EB56F040EB66FD7
:10499000000EAB6F040EAC6FABC5ADF5AE6F32C49D
:1049A000A9F5A95102E1100E12D0010EE66EE66AD9
:1049B000A90EE66E050EE66E010EE66EE66A70EC76
:1049C00039F0496E060EE15E49500501200EA86FD0
:1049D000E552E552E7CFD9FF1200D9CFE6FFE1CF8C
:1049E000D9FF020EE126000EDE6E040EDD6EFD0E16
:1049F000DB50E8244B6EFE0EDB50040DF3504B24CD
:104A0000040DF4CF4AF0D9CFE9FFDACFEAFFF35033
:104A1000EE264A50ED22DECFE9FFDDCFEAFFEF9E22
:104A2000FD0EDB500AE1FE0EEA6ADB34FE0BEA36CD
:104A3000E96EAF0EE926050E09D0FE0EEA6ADB34F8
:104A4000FE0BEA36E96EB50EE926050EEA22DECF48
:104A5000EEFFDDCFEDFFDECFE9FFDDCFEAFFEF9C1C
:104A6000DECFE9FFDDCFEAFF040EE926000EEA22E1
:104A7000EF8C020EE15C02E2E16AE552E16EE55282
:104A8000E7CFD9FF1200D9CFE6FFE1CFD9FF020E61
:104A9000E126FD0EDBA407D0E66AFE0EDBCFE6FFC3
:104AA0009CDFE552E552FD0EDBA208D0010EE66E5A
:104AB000FE0EDBCFE6FF91DFE552E552FE0EDB5046
:104AC0004A6A260F496E0F0E4A2249C0DEFF4AC0CD
:104AD000DDFFDECFE9FFDDCFEAFFFD0EDBCFEFFF2D
:104AE000020EE15C02E2E16AE552E16EE552E7CFD7
:104AF000D9FF1200D9CFE6FFE1CFD9FF020EE126A0
:104B0000FE0EDB5020E1ADC5E9FFAEC5EAFFEE5277
:104B1000400EEF6EADC5E9FFAEC5EAFF020EE92615
:104B2000000EEA22300EEE6E040EED6EADC5E9FF0A
:104B3000AEC5EAFF8C0EEF6EB5C5E9FFB6C5EAFF5C
:104B4000840EEF6E3BD0FD0EDB50E8244B6EFE0E64
:104B5000DB50040DF3504B24040DF3CF49F0F4CF98
:104B60004AF0000E4926040E4A2249C0DEFF4AC020
:104B7000DDFF840EDECFE9FFDDCFEAFFE850EF1264
:104B8000FD0EDB50E8244B6EFE0EDB50040DF3509F
:104B90004B24010F040DF3CF49F0F4CF4AF0000E7F
:104BA0004926040E4A2249C0DEFF4AC0DDFF840EBA
:104BB000DECFE9FFDDCFEAFFE850EF12020EE15C45
:104BC00002E2E16AE552E16EE552E7CFD9FF120059
:104BD000D9CFE6FFE1CFD9FF020EE126FD0EDB5073
:104BE0000AE0FE0EEA6ADB34FE0BEA36E96EB50E29
:104BF000E926050E09D0FE0EEA6ADB34FE0BEA3622
:104C0000E96EAF0EE926050EEA22EECFDEFFEDCF0C
:104C1000DDFFD9CFE9FFDACFEAFFEE50ED1003E177
:104C2000F36AF46A44D0DECFE9FFDDCFEAFF020E7B
:104C3000E926000EEA22FB0EDBCFEEFFFC0EDBCFF7
:104C4000EDFFDECFE9FFDDCFEAFFEE52FA0EDBCF5C
:104C5000EFFF400EDECFE9FFDDCFEAFFE850EF16B1
:104C6000880EDECFE9FFDDCFEAFFE850EF12FD0E40
:104C7000DB500AE0FE0EEA6ADB34FE0BEA36E96E30
:104C8000B50EE926050E09D0FE0EEA6ADB34FE0BEE
:104C9000EA36E96EAF0EE926050EEA22EF74DECFA2
:104CA00049F0DDCF4AF049C0F3FF4AC0F4FF020EDD
:104CB000E15C02E2E16AE552E16EE552E7CFD9FF3D
:104CC0001200D9CFE6FFE1CFD9FF65A84ED0FE0E86
:104CD000EA6ADB34FE0BEA36E96EB50EE926050E0C
:104CE000EA22EE50EFCFEAFFE96E400EEE16EE6AD2
:104CF000EE6AEE6AFE0EEA6ADB34FE0BEA36E96E15
:104D0000B50EE926050EEA22EE50EFCFEAFFE96E76
:104D1000EE7CFE0EEA6ADB34FE0BEA36E96EB50E77
:104D2000E926050EEA22EF74400E496EFE0EEA6A8D
:104D3000DB34FE0BEA36E96EB50EE926050EEA22F3
:104D4000EE50EFCFEAFFE96E4950EF16FE0EEA6A29
:104D5000DB34FE0BEA36E96EB50EE926050EEA22D3
:104D6000EE50EFCFEAFFE96EEF7CE552E7CFD9FFD7
:024D700012002F
:0E4D7200DACFE4FFE2CFDAFFE9CFE4FFEACFC9
:104D8000E4FFE6529EA076D19E908E0ECE6ECF6846
:104D90001850196E1A6A010E1B6E020E1E5C0EE18F
:104DA00002019451951104E002019407000E955BF5
:104DB00002019451951101E01B6A04D11E0401E027
:104DC00097D0105011100AE11250131007E114503F
:104DD000151004E11650171001E189D002019D5110
:104DE0000BE018A202D08D8001D08D9018A602D0C1
:104DF0008C8E01D08C9E0AD018A202D08C8001D05B
:104E00008C9018A602D08B8001D08B90105011107E
:104E10001DE000500824006E01500920016E000EB4
:104E2000D8800054800E015410E200C000F001C090
:104E300001F0000E005E800E015A010E1910196E6D
:104E4000010E1A6E1006000E115A1B6A1250131032
:104E50001DE002500A24026E03500B20036E000E68
:104E6000D8800254800E035410E202C002F003C046
:104E700003F0000E025E800E035A040E1910196E24
:104E8000010E1A6E1206000E135A1B6A1A502FE0FA
:104E900002019D5105E019B0898619B48A8004D0B9
:104EA00019B08C8219B48B8400000000000000004F
:104EB00000000000000000000000000000000000F2
:104EC00000000000000000000000000000000000E2
:104ED00000000000000000000000000000000201CF
:104EE0009D5103E089968A9002D08C928B946AD06F
:104EF000030E1E5C32E10501FE5105E0A1C27BF10B
:104F0000A2C27CF118D00E01005113E0B3CE7AFE9C
:104F1000B4CE7BFEB1CE4AFEB2CE4BFEB7CE32FE51
:104F20000E010251031104E1B1CE02FEB2CE03FE26
:104F300002D002019A6B899C02019451951104E000
:104F400002019407000E955B02019451951101E056
:104F50001B6A0201010EA36F35D0040E1E5C32E104
:104F60000501FE5105E09FC27BF1A0C27CF119D082
:104F70000E01005113E0B5CE7AFEB6CE7BFEAFCE69
:104F80004AFEB0CE4BFEB7CE32FE0E0102510311E7
:104F900004E1AFCE02FEB0CE03FE03D00201010E4B
:104FA0009A6F898C02019451951104E002019407D3
:104FB000000E955B02019451951101E01B6A0201FC
:104FC000A36B00D01B504AE01E6A1D5047E01C6ACC
:104FD000040E1C5C3AE21C50E96EEA6AD890E9368D
:104FE000EA36800EE926020EEA22EECF58F0EFCF25
:104FF00059F01C50E96EEA6AD890E936EA36080E94
:10500000E926000EEA2258C0EEFF59C0EDFF1C5001
:10501000E96EEA6AD890E936EA36880EE926020E89
:10502000EA22EECF58F0EFCF59F01C50E96EEA6A51
:10503000D890E936EA36100EE926000EEA2258C06A
:10504000EEFF59C0EDFF1C2AC3D790C218F091C2E1
:105050001EF092C294F293C295F21D6A8050800BAA
:1050600006E00201AA5106E08150040B03E10201AF
:10507000010EA96FE552E5CFEAFFE5CFE9FFE5CFE5
:10508000DAFF1100010E086E096A0A6E0B6A0C6ED7
:105090000D6A0E6E0F6A106A116A126A136A146A38
:1050A000156A166A176A1D6ACD92CD9ECD9CCD8A6F
:1050B000CD98CD96CD948E0ECE6ECF68CD809F804C
:1050C0009E909D80806A810E926E816A020E936E20
:1050D000F19E826A800E946E836A956A846A966AEB
:1050E0000F01FE0E486F1F0E496F89948C988D82B8
:1050F00089828C8C8C8A8D848B8289968D908A9003
:105100008C9E899C929C0201010E9A6F9D6F0501F5
:10511000FE6B0E01006F0201A36FA86BA46BA56B61
:10512000A66BA76BA96B9384F19EAA6FCB68800EC8
:10513000BB6EFC0ECA140009CA6E9D920F0152810B
:105140005293F00EBA140C09BA6E3F0EBA1400094D
:10515000BA6E0E010E0ECC6F9396CA841200D9CF90
:10516000E6FFE1CFD9FF030EE126DF6A010EDB6A1D
:10517000020EDB6AE66AD9CFE6FFDACFE6FF010E60
:10518000E66E4CEC1AF0E552E552E552E552E66A5D
:10519000D950010FE66E000EDA20E66E030EE66EC1
:1051A0004CEC1AF0E552E552E552E5522C5001E084
:1051B00014D1DF0446E1D950010FE96EDACFEAFFDE
:1051C000EE50ED1008E10E01006B0501FE6B0101D0
:1051D0007B6B7C6BEFD0D950010FE96EDACFEAFF21
:1051E000010EEE180FE1ED500DE10501010EFE6F0D
:1051F0000E01006B939201015A0501E0DBD0020E13
:105200005A6FD8D00501FE6B9392B3CEE6FFB4CEB1
:10521000E6FF040EE66EB1CEE6FFB2CEE6FF010E6B
:10522000E66EAEEC37F0496E060EE15E4950000EB8
:10523000E66EE66A010EE66E3EDBE552E552E552A9
:10524000B9D0020EDF5C15E1D950010FE96EDACF5B
:10525000EAFFEE50ED100AE10201010E9D6F9590FC
:10526000949095929494929A939AA4D002019D6BF3
:10527000A1D0040EDF5C07E1010EDBCFB1FE020E10
:10528000DBCFB2FE97D0050EDF5C07E1010EDBCF6E
:10529000AFFE020EDBCFB0FE8DD0060EDF5C1CE150
:1052A000D950010FE96EDACFEAFF720ED880EE54C2
:1052B0002E0EED540AE2720EF36E010EF3CFDBFFF9
:1052C0002E0EF36E020EF3CFDBFF010EDBCFA1F249
:1052D000020EDBCFA2F26ED0070EDF5C1CE1D950CC
:1052E000010FE96EDACFEAFF720ED880EE542E0E6F
:1052F000ED540AE2720EF36E010EF3CFDBFF2E0EB9
:10530000F36E020EF3CFDBFF010EDBCF9FF2020E36
:10531000DBCFA0F24FD0080EDF5C16E1D950010FB1
:10532000E96EDACFEAFF180ED880EE54000EED5485
:1053300007E2180EF36E010EF3CFDBFF020EDB6AFD
:10534000010EDBCFABFE36D0090EDF5C16E1D95083
:10535000010FE96EDACFEAFF060ED880EE54000E98
:10536000ED5407E2060EF36E010EF3CFDBFF020EE3
:10537000DB6A010EDBCFACFE1DD00A0EDF5C07E15D
:10538000010EDBCFB3FE020EDBCFB4FE0DD00B0E51
:10539000DF5C07E1010EDBCFB3FE020EDBCFB4FE14
:1053A00009D00C0EDF5C06E1010EDBCFB5FE020E6C
:1053B000DBCFB6FE0D0EDF5C0EE1D950010FE96EBA
:1053C000DACFEAFFEE50ED1004E00201010EAA6F01
:1053D00002D00201AA6B0FEC12F0030EE15C02E2B4
:1053E000E16AE552E16EE552E7CFD9FF1200D9CF6D
:1053F000E6FFE1CFD9FF0A0EE126020EDB6A030EBB
:10540000DB6A040EDB6A050EDB6A060EDB6A070E3A
:10541000DB6A080EDB6A090EDB6AE66AD9CFE6FFB3
:10542000DACFE6FF030EE66E4CEC1AF0E552E552D9
:10543000E552E552E66AD950020FE66E000EDA2018
:10544000E66E020EE66E4CEC1AF0E552E552E552BD
:10545000E552010EE66ED950040FE66E000EDA201A
:10546000E66E020EE66E4CEC1AF0E552E552E5529D
:10547000E5522C5023E1080EDBCFE6FF090EDBCF0F
:10548000E6FF060EDBCFE6FF070EDBCFE6FF040EDE
:10549000DBCFE6FF050EDBCFE6FF020EDBCFE6FF3C
:1054A000030EDBCFE6FFDECFE6FFDDCFE6FF10D851
:1054B000496E0A0EE15E49500FEC12F00A0EE15CF3
:1054C00002E2E16AE552E16EE552E7CFD9FF120050
:1054D000D9CFE6FFE1CFD9FF1D50FEE1D950FB0F38
:1054E000E96EFF0EDA20EA6EEE50ED102EE1D95093
:1054F000F90FE96EFF0EDA20EA6EEE50ED1025E1AD
:10550000D950F70FE96EFF0EDA20EA6EEE50ED107B
:105510001CE1D950F50FE96EFF0EDA20EA6EEE506D
:10552000ED1013E10201020E916F190E3D6E3E6AFD
:10553000FD0EDBCF42F0FE0EDBCF43F0CFEC3AF0B6
:105540003BC092F23CC093F2EBD0010E0201926F8D
:10555000936B906B89948C98FB0EDBCF49F0FC0E1B
:10556000DBCF4AF0800E4A1413E0020E9011906FC8
:105570003D683E68FB0EDBCF42F0FC0EDBCF43F014
:10558000A2EC3AF0FB0E3BC0DBFFFC0E3CC0DBFFA5
:10559000F90EDBCF49F0FA0EDBCF4AF00001800EA6
:1055A0004A1414E0080E02019011906F3D683E68A5
:1055B000F90EDBCF42F0FA0EDBCF43F0A2EC3AF06B
:1055C000F90E3BC0DBFFFA0E3CC0DBFFFD0EDBCF6C
:1055D0004DF0FE0EDBCF4EF04F6A506A190E406E52
:1055E000416A426A436A4DC03BF04EC03CF04FC036
:1055F0003DF050C03EF077EC3BF037C04DF038C086
:105600004EF039C04FF03AC050F0FB0EDBCF49F0FE
:10561000FC0EDBCF4AF04B6A4C6A4AAE02D04B68B4
:105620004C680F0ED89049364A364B364C36E80651
:10563000F9E149C03BF04AC03CF04BC03DF04CC0E2
:105640003EF04DC040F04EC041F04FC042F050C05F
:1056500043F0D5EC3BF03BC080F23CC081F2010E40
:1056600002018027000E8123FB0EDBCF88F2FC0EA7
:10567000DBCF89F2FD0EDBCF4DF0FE0EDBCF4EF01F
:105680004F6A506A190E406E416A426A436A4DC0C1
:105690003BF04EC03CF04FC03DF050C03EF077ECC8
:1056A0003BF037C04DF038C04EF039C04FF03AC033
:1056B00050F0F90EDBCF49F0FA0EDBCF4AF04B6A1F
:1056C0004C6A4AAE02D04B684C680F0ED8904936EF
:1056D0004A364B364C36E806F9E149C03BF04AC041
:1056E0003CF04BC03DF04CC03EF04DC040F04EC0D1
:1056F00041F04FC042F050C043F0D5EC3BF03BC00E
:1057000082F23CC083F2010E02018227000E832345
:10571000F90EDBCF8AF2FA0EDBCF8BF2010E916F1E
:10572000010E1D6EE552E7CFD9FF1200A3C249F06A
:105730004A6A49BE4A6849C0E6FF4AC0E6FF460ECB
:105740004B6E700E4C6E4D6A4BC0E6FFE66E4DC060
:10575000E6FF56EC3AF04E6E050EE15E4E500FEF4E
:1057600012F0D9CFE6FFE1CFD9FF020EE126F40E09
:10577000DE6E010EDD6EE66ED9CFE6FFDACFE6FF14
:10578000030EE66E4CEC1AF0E552E552E552E55296
:105790002C5015E10201A30506E1DECFE6FFDDCFC7
:1057A000E6FFE66A06D0DECFE6FFDDCFE6FF010EBC
:1057B000E66E81D8E552E552E5520FEC12F0020E8A
:1057C000E15C02E2E16AE552E16EE552E7CFD9FF22
:1057D0001200D9CFE6FFE1CFD9FF040EE126DF6A40
:1057E000010EDB6A020EDB6A010EF36E030EF3CFCD
:1057F000DBFFE66AD9CFE6FFDACFE6FF010EE66E01
:105800004CEC1AF0E552E552E552E552010EE66E17
:10581000D950010FE66E000EDA20E66E030EE66E3A
:105820004CEC1AF0E552E552E552E552010EE66EF7
:10583000D950030FE66E000EDA20E66E010EE66E1A
:105840004CEC1AF0E552E552E552E5522C5029E1B4
:10585000030EDB50070805E2010EF36E030EF3CFD3
:10586000DBFF030EDB50030F0E01B76F010EF36E6B
:10587000030EDB5004E0D890F336E806FCE1F35069
:10588000F31C9314936E010EDBCFE6FF020EDBCF09
:10589000E6FFDFCFE6FF0FD8E552E552E5520FEC09
:1058A00012F0040EE15C02E2E16AE552E16EE552BB
:1058B000E7CFD9FF1200D9CFE6FFE1CFD9FF1D50C6
:1058C000FEE1FE0EDB0403E10201030E02D0020141
:1058D000040E916F190E3D6E3E6AFC0EDBCF42F056
:1058E000FD0EDBCF43F0CFEC3AF03BC092F23CC070
:1058F00093F2010E1D6EE552E7CFD9FF1200D9CF0A
:10590000E6FFE1CFD9FF050EE126E66AD9CFE6FF33
:10591000DACFE6FF010EE66E4CEC1AF0E552E552E6
:10592000E552E552E76E040EE7CFDBFFDB5025E1E1
:105930002C5066E102019D511AE0DF50000815E28B
:105940008994DF0402E18D828982020EDF5C02E12C
:105950008D928982030EDF5C02E18D828992040EB2
:10596000DF5C0BE18D92899208D0898406D0DF50EC
:10597000000802E2899A01D0898A010EE66ED950A8
:10598000010FE66E000EDA20E66E010EE66E4CECBC
:105990001AF0E552E552E552E552E76E040EE7CF04
:1059A000DBFFDB502BE12C502BE102019D511FE06E
:1059B000010EDB50000819E28C98010EDB0402E1B5
:1059C0008C8C8C8A010EDB50020802E18C9C8C8A44
:1059D000010EDB50030802E18C8C8C9A010EDB5027
:1059E00004080CE18C9C8C9A09D08C8807D0010E9D
:1059F000DB50000802E28A9A01D08A8A0FEC12F08A
:105A0000050EE15C02E2E16AE552E16EE552E7CFA4
:105A1000D9FF1200FE0E0201A45DFF0EA559FF0E74
:105A2000A659FF0EA75905E2A42B000EA523A62315
:105A3000A7230FEF12F00201A451A511A611A7117F
:105A400005E0A407000EA55BA65BA75B0FEF12F0B5
:105A5000D9CFE6FFE1CFD9FF050EE126E66AD9CF1F
:105A6000E6FFDACFE6FF070EE66E4CEC1AF0E552E1
:105A7000E552E552E552E76E040EE7CFDBFFDB505F
:105A80000BE1DFCFA4F2010EDBCFA5F2020EDBCFDC
:105A9000A6F2030EDBCFA7F20FEC12F0050EE15CCD
:105AA00002E2E16AE552E16EE552E7CFD9FF12006A
:105AB000A4C2E6FFA5C2E6FFA6C2E6FFA7C2E6FFB4
:105AC0003D0E496E700E4A6E4B6A49C0E6FFE66EA7
:105AD0004BC0E6FF56EC3AF04C6E070EE15E4C50C0
:105AE0000FEF12F0E66AA80EE66E020EE66E010EE9
:105AF000E66E4CEC1AF0E552E552E552E5522C50B8
:105B000001E012000FEF12F0A8C249F04A6A49BE44
:105B10004A6849C0E6FF4AC0E6FF360E4B6E700E7B
:105B20004C6E4D6A4BC0E6FFE66E4DC0E6FF56EC8C
:105B30003AF04E6E050EE15E4E500FEF12F0A9C224
:105B400049F04A6A49BE4A6849C0E6FF4AC0E6FFD2
:105B5000300E4B6E700E4C6E4D6A4BC0E6FFE66E1B
:105B60004DC0E6FF56EC3AF04E6E050EE15E4E502B
:105B70000201A96B0FEF12F0D9CFE6FFE1CFD9FFF9
:105B8000040EE126DE6ADD6A020EDB6A030EDB6AC2
:105B9000C26AA40EC16E9E9C9F9CC28002010A0E26
:105BA000AB6FAB51FEE1C282C2B2FED7C4504C6EA5
:105BB0004B6AC3504B24496E000E4C2049C0DEFF97
:105BC000DD6E2D0EC26E02010A0EAB6FAB51FEE10F
:105BD000C282C2B2FED7C4504C6E4B6AC3500001A1
:105BE0004B24496E000E4C204A6E020E49C0DBFF6A
:105BF000030E4AC0DBFF020EDBCFE6FF030EDBCF56
:105C0000E6FFDECFE6FFDDCFE6FF240E496E700E25
:105C10004A6E4B6A49C0E6FFE66E4BC0E6FF56ECA3
:105C20003AF04C6E070EE15E4C500FEC12F0040E91
:105C3000E15C02E2E16AE552E16EE552E7CFD9FFAD
:105C40001200D9CFE6FFE1CFD9FF030EE126DF6ACC
:105C5000010EDB6A040EF36E020EF3CFDBFFE66A81
:105C6000D9CFE6FFDACFE6FF010EE66E4CEC1AF074
:105C7000E552E552E552E552010EE66ED950010FAC
:105C8000E66E000EDA20E66E030EE66E4CEC1AF0BD
:105C9000E552E552E552E5522C503CE1D950010F56
:105CA000E96EDACFEAFFFF0ED880EE54030EED5412
:105CB00006E3010EDBCFACF2020EDBCFADF2DF501C
:105CC00023E0ACC249F0ADC24AF0D8904A32493222
:105CD000D8904A3249324950BB6EACC24BF0ADC28B
:105CE0004CF0040ED8904B364C36E804FBE1300EF5
:105CF0004B16000E4C16CF0EBA1400014B10496E15
:105D00004CC04AF0E85003D0BB6ACF0EBA14BA6E4A
:105D10000FEC12F0030EE15C02E2E16AE552E16E83
:0C5D2000E552E7CFD9FF1200120012007C
:045D2C00D2EC33F092
:105D3000FB0EDBCFF3FFDB06F35000090AE020EC9B
:105D400034F0FA0E8BEC34F0F3E14A1CF1E1010E71
:105D500001D0000E01EF34F0D2EC33F03B0EE12421
:105D600002E3E168E652E16E010EDB6A020EDB6AD5
:105D7000F90EDBCFF6FFFA0EDBCFF7FFFB0EDBCF22
:105D8000F8FF0800F550DF6EDF5002E125EF33F039
:105D9000250EDF5C02E018EF33F0030EDB6A040E21
:105DA000DB6A050EDB6A060EDB6A070EDB6A3AEC7D
:105DB00033F02D0EDF5C0CE02B0EDF5C09E0200ED3
:105DC000DF5C06E0230EDF5C03E0300EDF5C1AE1EF
:105DD000DF50300A14E0130A0FE0030A0AE00B0A4E
:105DE00005E0060AE4E1030EDB80E1D7030EDB8267
:105DF000DED7030EDB84DBD7030EDB86D8D7030E9A
:105E0000DB88D5D72A0EDF5C1BE136EC33F084EC5F
:105E100033F010E0030EDB803D683E68130EDBCFED
:105E200042F0140EDBCF43F0A2EC3AF0040E3BC07C
:105E3000DBFF03D0130E6DEC33F03AEC33F00BD0F4
:105E4000090EDB6ADBEC33F003E04FEC34F0FAD7F9
:105E5000090E6DEC33F0030EDBB0DB982E0EDF5C29
:105E60001BE13AEC33F02A0EDF5C0BE136EC33F049
:105E700084EC33F003E1130EBFEC33F03AEC33F073
:105E80000BD0090EDB6ADBEC33F003E04FEC34F0AF
:105E9000FAD7090EBFEC33F0680EDF5C07E13AEC8D
:105EA00033F0680EDF5C1DE1030E18D0740EDF5C6A
:105EB00017E07A0EDF5C14E0480EDF5C06E0540E5B
:105EC000DF5C03E05A0EDF5C02E1020E07D06C0ECD
:105ED000DF5C03E06A0EDF5C04E1010E12EC34F0DB
:105EE000C9DBDF506E0A01E17FD31E0A01E192D1C6
:105EF000200A01E18FD13F0A01E149D11A0A01E1EB
:105F000046D10D0A01E143D1200A01E140D13A0A0C
:105F100001E13DD1200A01E13AD1260A01E135D162
:105F20000D0A01E132D11A0A01E1D9D0200A4AE072
:105F3000300A1FE0460A0EE0250A01E083D3D9505B
:105F4000F90FE96EFF0EDA20EA6E010EEE5E000E2A
:105F5000EE5AEE5A20EC34F0250EE66E95DB03E1A6
:105F60004A1C01E169D31CEC34F001E26BD3DB2A5B
:105F700069D3080EDB6A040EDB50010806E2040E4A
:105F8000DB04E4EC33F0DB508BDB080EDB5009E084
:105F9000030EDB50010B05E172DB01E04DD3080E6F
:105FA000DB6A64DBEFCFDFFF94EC34F003E14A1CE3
:105FB00001E142D31CEC34F001E3DB2A60DB01E1B8
:105FC00041D33AD3070EDB5002080FE160EC34F006
:105FD000030E27EC34F00E0EEECFDBFF0F0EEECFEC
:105FE000DBFF100EEECFDBFF20D0F70EDBCF4CF047
:105FF000F80EDBCF4DF0020E4C5E000E4D5AF70E40
:106000004CC0DBFFF80E4DC0DBFF4CC0E9FF4DC0BC
:10601000EAFF17EC34F04B6A0E0E49C0DBFF0F0E9F
:106020004AC0DBFF100E4BC0DBFF0E0EDBCFE6FFDE
:106030000F0EDBCFE6FF100EDBCFE6FF31EC3AF0C0
:10604000E552E552E552130E3CC0DBFF140E3DC095
:10605000DBFF060EDB5005E0130E5BEC34F001E2D3
:106060006ADB7FEC34F002E2130E37DB42EC34F0F3
:1060700006E0040E5BEC34F002E2050E2EDB030EAC
:10608000DBB005D0FCDA01E0D7D2080EDB6A090EDE
:10609000DB6A0E0EDBCFF6FF0F0EDBCFF7FF100E25
:1060A000DBCFF8FF0800F550DF6EDF5014E085EC21
:1060B00034F011E294EC34F003E14A1C01E1BCD26B
:1060C000BBDB01E3DB2A090EDB2AD9500E0FE96E98
:1060D000000ECBDBE7D7D3DA01E1B4D2ADD2C6DA1A
:1060E000110EEECFDBFF120EEDCFDBFF110EDBCF7B
:1060F000E6FF120EDBCFE6FF23EC3AF0E552E55265
:10610000130EF3CFDBFF140EF4CFDBFF060EDB50D4
:1061100004E0130ED0DB01E20EDB7FEC34F002E290
:10612000130EDBDAAFDB05E0040EC5DB02E2050E81
:10613000D4DA030EDBB005D0A2DA01E07DD2080E7E
:10614000DB6A090EDB6A110EDBCFE9FF120EDBCF33
:10615000EAFFEFCFDFFFDF5014E0D7DB12E2E4DB32
:1061600003E14A1C01E168D267DB01E3DB2A090E87
:10617000DB2A110EDB2ADBCFE9FF120EE8E3DB2A74
:10618000E6D77DDA01E15ED257D2030EDB8E070E31
:10619000DB0410E195DB040E5ADB0A0EEECFDBFFC9
:1061A0000B0EEECFDBFF0C0EEECFDBFF0D0EEECFB6
:1061B000DBFF6CD0070EDB5003082CE1030EDBAED7
:1061C0000DD0B2DA020E76DAEFCF49F04A6A4B6AA6
:1061D0004C6A49AE39D04A684B6835D0F70EDBCFF0
:1061E0004AF0F80EDBCF4BF0020E4A5E000E4B5A1F
:1061F000F70E4AC0DBFFF80E4BC0DBFF4AC0E9FFD9
:106200004BC0EAFFEFCF49F00A0E49C0DBFF0B0E8F
:10621000DB6A38D0070EDB50020809E1030EDBAE63
:1062200004D059DB4BAE10D00ED055DB0DD0030E91
:10623000DBAE12D079DA020E3DDAF9DA4B6A4C6A3B
:106240004AAE02D04B684C68E2DA0C0E4BC0DBFF62
:106250000D0E4CC0DBFF1AD0F70EDBCF4BF0F80E63
:10626000DBCF4CF0020E4B5E000E4C5AF70E4BC0CB
:10627000DBFFF80E4CC0DBFF4BC0E9FF4CC0EAFF70
:10628000D6DAC5DA0C0EDB6A0D0EDB6A060EDB50C1
:1062900005E1010EF36E050EF3CFDBFF150EDB6A91
:1062A000160EDB6AD950370F496E000EDA204A6E9F
:1062B000390E49C0DBFF3A0E4AC0DBFF380EDB6AFD
:1062C000080EDB6A0A0EAEDADF50780A12E0200A06
:1062D00010E0280A0CE0200A0AE03F0A06E00D0A56
:1062E00002E0200A08E1020E05D0080E03D0080ED5
:1062F000DF26100E97DA030EDBBE02D0DB92DB94B2
:10630000DB50800B24E08ADAD890030EEB50000AB1
:1063100008E6000EEE5C000EEE58000EEE58000E81
:10632000EE5815E213DA406841684268436877EC3A
:106330003BF00A0E37C0DBFF0B0E38C0DBFF0C0E44
:1063400039C0DBFF0D0E3AC0DBFF2D0E08D0030E67
:10635000DBA202D02B0E03D0DBA408D0200EF36EFC
:10636000170EF3CFDBFF150EDB2A02D0170EDB6A08
:10637000050EDB5003E1B7D901E189D0760E496EF5
:10638000780E4A6E000E4B6E070EDBCF4CF04D6A56
:106390004E6A4F6A4CC040F04DC041F04EC042F0D2
:1063A0004FC043F0D3D9D5EC3BF049503724F36EBE
:1063B0004A503820F46E4B503920F86EF4CFF7FF76
:1063C000F3CFF6FF0800090EF5CFDBFF580EDF5CB8
:1063D0000FE1610EF36E090E7BD90AE3200E496EC0
:1063E000090EDBCFE7FF4950E75E090EE7CFDBFF81
:1063F000070EDBCF49F04A6A4B6A4C6A0FDA49C094
:1064000040F04AC041F04BC042F04CC043F0EECFE8
:106410003BF0EECF3CF0EECF3DF0EFCF3EF0D5ECD1
:106420003BF03EC0EDFF3DC0EDFF3CC0EDFF3BC08B
:10643000EFFF390EDBCFE9FFDB063A0EDBCFEAFFD9
:1064400001E2DB06090EDBCFEFFF150EDB2A4BD98D
:1064500095E1030EDBA61DD06F0EDF5C06E1C1D90E
:1064600018E3150EDB285BDA14D0780EDF5C09E048
:10647000580EDF5C06E0620EDF5C03E0420EDF5C7C
:1064800008E1020EF36E160EF3CFDBFF02D0150EFD
:10649000DB6A030EDB50100B0EE0040EDBCF49F07D
:1064A000050EDB50D880495406E2060EDB5003E1AE
:1064B000040EDB5034DA95D90AE2050EDBCFE7FF94
:1064C000150EDB50E75E050EE7CFDBFF02D0050EB1
:1064D000DB6A040EDBCF49F0160E45D9D88049544B
:1064E00014E2160EDBCFE6FF150EDBCFE6FF040E3F
:1064F000DBCFE6FF050EDB50E552E75CE552D880C6
:10650000E754E552D880E7545FD9030EDB50010B06
:106510000BE1080EDB5008E0B2D801E08DD0080E88
:10652000DB50BED8080EDB6A170EDB5007E088D9B7
:10653000170EF1D903E14A1C01E17ED0160EDB50A3
:1065400016E07ED9300EE66E9FD802E14A1C74E058
:1065500077D9DFCFE6FF35EC3BF0E552E552E55267
:10656000F4CF4AF00001F31C02E14A1C65E0050E7D
:10657000DBCF49F0160EDB50D880495409E2050EF6
:10658000DBCFE7FF160EDB50E75E050EE7CFDBFF44
:10659000300EE66E050ECBD94FE1390EDB2ADBCF8C
:1065A000E9FF3A0E01E3DB2ADBCFEAFF090EEFCF6A
:1065B000DBFFDB500EE044D9090EADD902E14A1CE5
:1065C0003BE0390EDB2ADBCFE9FF3A0EEDE3DB2AB5
:1065D000EBD755D831E1160EDBCFE6FF080EC3D856
:1065E000E552E7245DD82ED0070EDB50030A1CE0ED
:1065F000010A14E0030A07E07BD9DBCFEEFF020EAD
:10660000DBCFEDFF1FD0F5D84E6A4CAE02D04D68FF
:106610004E682CD8BCD84EC0EEFF14D0EAD84CBE81
:106620004D6824D8B4D80ED063D9DBCFEFFF0AD0A1
:106630007BD905E14A1C03E1F368F46810D0FCD86B
:1066400001E3DB2A79D9C1EF2EF0010EDBCF49F04F
:10665000020EDBCF4AF049C0F3FF4AC0F4FF3B0E05
:10666000E15C02E2E16AE552E16ECBD029D9020E8B
:1066700027EF34F061D90800F550DF6E1200200ECC
:10668000E66E080E97EF34F035EC3BF0E552E5523C
:10669000E552F3CF49F0F4CF4AF00001F31C1200A9
:1066A000496E4A6AD950010F4DD94950EE264A50D9
:1066B000ED2212004D5E000E4E5AF70E4DC0DBFF6C
:1066C000F80E4EC0DBFF4DC0E9FF4EC0EAFF1200DE
:1066D000DBCFF4FFF350F45C1200DB50E76E040EE6
:1066E000E7CFDBFF12000A0EDBCF49F00B0EDBCF4A
:1066F0004AF00C0EDBCF4BF00D0EDBCF4CF04950C7
:106700004A104B104C101200130EEECFDBFF140E8C
:10671000EDCFDBFF130EDBCF49F0140EDBCF4AF0D9
:106720000001800E4A141200F70EDBCF4DF0F80E78
:10673000DBCF4EF01200050EDB50E66ED950130F82
:1067400001D9E552E750EE6EED6A12000A0EDBCF7A
:106750003BF00B0EDBCF3CF00C0EDBCF3DF00D0E13
:10676000DBCF3EF01200DBCFE6FF150EDBCFE6FFFE
:10677000050EDB50E552E724E552E7241200DB501A
:10678000CED8010EF36E060EF3CFDBFF1200EE50F3
:10679000EFCFEAFFE96E4BC0EEFF4CC0EEFF4DC0FD
:1067A000EEFF1200D9CFE6FFDACFE6FFE1CFD9FF47
:1067B000E2CFDAFF1200DFCFE6FFE66AC3EC3BF080
:1067C000E552E552F3501200E76E080EE7CFDBFF0B
:1067D0001200EECF49F0EECF4AF0EFCF4BF04C6A0B
:1067E0001200050EDBCF49F0150EDB50D88049545E
:1067F0001200010EDBCF4BF0020EDBCF4CF04D6AE6
:106800001200E552E5CFDAFFE7CFD9FF12000A0EFA
:1068100049C0DBFF0B0E4AC0DBFF1200D9500A0F44
:10682000A2EF34F0F36E070EF3CFDBFF1200EECFD2
:1068300049F0EFCF4AF01200010EDB2A020E1200DF
:10684000FC0EDBCFE6FFFD0EDBCFE6FF1200495E5C
:10685000000E4A5AF70E49C0DBFFF80E4AC0DBFFB4
:1068600049C0E9FF4AC0EAFF1200DA20EA6EEF2AC7
:10687000EECFF6FF000EEF22EECFF7FFEF22EECFC6
:10688000F8FF1200040EDBCFE6FF130EDB50E552DB
:10689000E75C9ADFDB5004DF060EDB501200090EC6
:1068A000DB500A0DF350DF24D00FE76E090EE7CF5F
:1068B000DBFF3AEF33F0DB50F36E050E68EF33F099
:1068C000F70EDBCF49F0F80EDBCF4AF01200DFCF36
:1068D000E6FF44EF33F028DF030EECDEE9EF33F0A0
:1068E00096EC2EF0E552E552E552E5520009120011
:1068F000BDDEEE50EFCFEAFFE96E010E1200130E7F
:10690000DB50F36E040E68EF33F0040EDB50F36ED1
:10691000090E68EF33F0DBCFE6FF44EF33F0E76EAC
:10692000050EE7CFDBFF12008BDF67EF34F0DBCF24
:10693000E6FF86DF70EF34F0D950F90FE96EFF0EF5
:0E69400035EF34F0E96E000EDA20EA6E120038
:02694E00040142
:1069500030511F0B010801E012003051600BE8427A
:10696000E842E842E842E842010801E012003451FE
:1069700003E0340501E012003151220A31E0030A3C
:1069800024E0010A15E0210A0DE0010A01E01200ED
:106990000501A00EBD6F050EBE6F080EC06FC16B66
:1069A000BF8121D00501A00EBD6F050EBE6F1BD0AB
:1069B00036C4C5F537C4C6F50501880EC26F050E8D
:1069C000C36FC76BC86BC48F12000501880EBD6F03
:1069D000050EBE6F070EC06FC16BC10EBF6F1200F8
:1069E00032C49BF50501BF8F12000501886B4B0E69
:1069F000896F8A6B8B6B8C6B8D6B080E8E6F8F6BB8
:106A00001A0EE66E010EE66E43EC25F0E552E552F5
:106A10001E0EE66E020EE66E43EC25F0E552E552E0
:106A2000400EE66E080EE66E050EE66EE66A020E93
:106A3000E66EE8EC25F0496E050EE15E4950F3CFB5
:106A400097F5F4CF98F50501996B9A6B906B12004E
:106A5000D9CFE6FFE1CFD9FF05018F6B9751981190
:106A600002E1000E08D097C5E9FF98C5EAFFEF5094
:106A7000800B01E0010E000945E1FC0EDBCF49F07F
:106A800097C5E9FF98C5EAFFEE52EF50D880495408
:106A900008E297C5E9FF98C5EAFFEE52FC0EEFCF7A
:106AA000DBFF8F6BFC0EDB508F5D19E28F51EA6AC2
:106AB000080FE96E050EEA22EF50E66E8F51E76E81
:106AC000FD0EDBCFE9FFFE0EDBCFEAFFE750E92644
:106AD000000EEA22E552E750EF6E8F2BE3D7400E0F
:106AE000E66E080EE66E050EE66EE66A020EE66ECD
:106AF000E8EC25F0496E050EE15E4950F3CF97F5BD
:106B0000F4CF98F505018F51E552E7CFD9FF120078
:106B1000D9CFE6FFE1CFD9FF050190510CE1FD0E81
:106B2000DBCF91F5FE0EDBCF92F5FC0EDBCF95F5BA
:106B3000010E966F906FE552E7CFD9FF1200D9CFC3
:106B4000E6FFE1CFD9FF030EE126050190512DE1CB
:106B5000DF6AFD0EDBCF3DF0FE0EDBCF3EF0DE52F6
:106B60003DC0DEFF3EC0DDFFDD52DF2ADF50496E53
:106B70004A6AFF0E491802E14A500BE0010EDBCFD2
:106B8000E9FFDB2A020EDBCFEAFF01E3DB2AEF504D
:106B9000ECE1FD0EDBCF91F5FE0EDBCF92F5DFCF02
:106BA00095F50501010E966F906F030EE15C02E210
:106BB000E16AE552E16EE552E7CFD9FF1200D9CF85
:106BC000E6FFE1CFD9FF030EE126050190512EE14A
:106BD000DF6AFD0EDBCF3DF0FE0EDBCF3EF0DE5276
:106BE0003DC0DEFF3EC0DDFFDD52DF2ADF50496ED3
:106BF0004A6AFF0E491802E14A500CE0010EDBCF51
:106C0000F6FFDB2A020EDBCFF7FF01E3DB2A0800E9
:106C1000F550EBE1FD0EDBCF91F5FE0EDBCF92F5EB
:106C2000DFCF95F50501966B010E906F030EE15CC9
:106C300002E2E16AE552E16EE552E7CFD9FF1200C8
:106C4000D9CFE6FFE1CFD9FF020EE1260501995128
:106C50009A1102E1000E08D099C5E9FF9AC5EAFF32
:106C6000EF50800B01E0010E000901E084D0030E1B
:106C7000905D01E1906B905101E17DD0020E905D3D
:106C800016E1E66A000EE66EE66A010EE66E020E98
:106C9000E66EE8EC25F0496E050EE15E4950F3CF53
:106CA00099F5F4CF9AF50501030E906F64D0900525
:106CB00062E1400E496E4A6A9551495C000E4A589D
:106CC00003E2400EDF6E02D095C5DFFFDF50955D19
:106CD000956F480E936F050E946F010EDFCFDBFFAB
:106CE000965116E1010EDB5028E091C5F6FF92C5E2
:106CF000F7FF0800F55093C5E9FF94C5EAFFEF6E72
:106D0000932B000E9423912B9223010EDB06EAD7DE
:106D1000010EDB5012E091C5E9FF92C5EAFFEF508A
:106D200093C5E9FF94C5EAFFEF6E932B000E942301
:106D3000912B9223010EDB06EBD70501955107E15C
:106D4000400EDF5C02E1020E01D0030E906FDFCF38
:106D5000E6FF480EE66E050EE66E010EE66E020ECA
:106D6000E66EE8EC25F0496E050EE15E4950F3CF82
:106D700099F5F4CF9AF5020EE15C02E2E16AE55280
:0A6D8000E16EE552E7CFD9FF1200E3
:066D8A00D9CFE6FFE1CFC6
:106D9000D9FFE6520E01006B016BAA6BDF6A180E79
:106DA000DF5C2AE2EA6ADF34FE0BEA36E96E020EA5
:106DB000E9260E0EEA22EE6AED6ADF50EA6A320F29
:106DC000E96E0E0EEA22EF6AEA6ADF34FE0BEA365B
:106DD000E96E4A0EE9260E0EEA22EE6AED6AEA6ACA
:106DE000DF34FE0BEA36E96E7A0EE9260E0EEA2251
:106DF000EE6AED6ADF2AD3D70E01C60EAD6F0E0E16
:106E0000AE6F3F0E79140009796ECF0E7914000928
:106E1000796E79827B6A7A6A79900F0152815293F6
:106E2000F00EB4140909B46E0E01070EAB6F030E19
:106E3000AC6FE00EB16F2E0EB26F800EAF6F3E0ED4
:106E4000B06F040EB76F93940501FE6B93920E0121
:106E5000010E006F900EB36F010EB46F900EB56F00
:106E6000010EB66FE552E552E7CFD9FF1200D9CF38
:106E7000E6FFE1CFD9FF050EE126DF6A010EDB6AEE
:106E8000020EDB6A030EDB6A040EDB6AE66AD9CF08
:106E9000E6FFDACFE6FF010EE66E4CEC1AF0E552A3
:106EA000E552E552E552010EE66ED950010FE66E4D
:106EB000000EDA20E66E030EE66E4CEC1AF0E55298
:106EC000E552E552E552010EE66ED950030FE66E2B
:106ED000000EDA20E66E010EE66E4CEC1AF0E5527A
:106EE000E552E552E552010EE66ED950040FE66E0A
:106EF000000EDA20E66E030EE66E4CEC1AF0E55258
:106F0000E552E552E5522C501FE1DF50180804E32A
:106F1000030EDB50180802E22C8C16D0040EDBCFD7
:106F2000E6FFE66A030EDBCFE6FF010EDBCFE6FFEE
:106F3000020EDBCFE6FFDFCFE6FF10D8496E060E6C
:106F4000E15E49500FEC12F0050EE15C02E2E16AED
:106F5000E552E16EE552E7CFD9FF1200D9CFE6FF47
:106F6000E1CFD9FFFE0EDB5003E10E01006B56D0DE
:106F7000FE0EDB50180852E3FB0EDB5018084EE300
:106F80000E01010E006FFE0EDB04E96EEA6AD89076
:106F9000E936EA367A0EE9260E0EEA22F90EDBCF42
:106FA000EEFFFA0EDBCFEDFFFE0EDB04E96EEA6AC0
:106FB000D890E936EA364A0EE9260E0EEA22FC0E91
:106FC000DBCFEEFFFD0EDBCFEDFFFE0EDB04EA6A4A
:106FD000320FE96E0E0EEA22FB0EDBCFEFFFFE0E44
:106FE000DB04E96EEA6AD890E936EA36020EE92651
:106FF0000E0EEA22EE50ED1011E1FE0EDB04E96EFA
:10700000EA6AD890E936EA36020EE9260E0EEA223E
:10701000FC0EDBCFEEFFFD0EDBCFEDFFE552E7CF41
:04702000D9FF120082
:0C702400253034692C253034690D0A0039
:107030002531690D0A00253033690D0A00253031EC
:10704000306C750D0A0025640A0D00537461747567
:10705000733D25690D0A002135204572723A204E94
:1070600065656420636F6D6D61206E6578742C209A
:10707000666F756E643A20272563270D0A005061FC
:1070800072616D383D25630D0A00506172616D3784
:107090003D25630D0A00506172616D363D256C75AA
:1070A0000D0A00506172616D353D256C640D0A005A
:1070B000506172616D343D25750D0A005061726139
:1070C0006D333D25640D0A00506172616D323D25BE
:1070D000640D0A00506172616D313D25640D0A0036
:1070E00050492C2531750D0A004D522C2530337531
:1070F0000D0A002C25303475004100492C25303311
:10710000692C253033692C253033692C25303369BF
:107110002C253033690D0A002138204572723A203F
:10712000556E6B6E6F776E20636F6D6D616E642050
:1071300027256325633A253258253258270D0A0042
:107140002138204572723A20556E6B6E6F776E2033
:10715000636F6D6D616E64202725633A2532582771
:107160000D0A002137204572723A20457874726109
:10717000207061726D617465720D0A0021362045C0
:1071800072723A20496E76616C6964207061726136
:107190006D7465722076616C75650D0A002134206E
:1071A0004572723A204D697373696E67207061721F
:1071B000616D657465722873290D0A0021332045BD
:1071C00072723A20525820427566666572206F7658
:1071D000657272756E0D0A002132204572723A2076
:1071E000545820427566666572206F7665727275B6
:1071F0006E0D0A002131204572723A2043616E27DC
:10720000742073746570207468617420666173748F
:107210000D0A002130200D0A002008002573001BF4
:0B7220005B421B5B314B1B5B304700E7
:04722C0005D82FEC66
:107230001EF00BEC0DF0FBD7D9CFE6FFE1CFD9FF65
:10724000020EE1260F0148694969600ED36E9B8CDE
:10725000580EDE6E020EDD6EDFCF49F0DF06010E46
:10726000DBCF4AF001E2DB0649504A10F5E14AEC77
:107270000CF09FEC1DF0020EE15C02E2E16AE552C7
:10728000E16EE552E7CFD9FF1200120012001200A2
:107290001200A7EF34F01200F5EF34F00501CB0532
:1072A0001EE10501CC051BE1F1DF65920501CC6B08
:1072B0000101100EFD6F0E0EFE6FFD07000EFE5B4E
:1072C000FD51FE11FAE16584080EFD6F070EFE6F99
:1072D000FD07000EFE5BFD51FE11FAE16594120000
:1072E000D9CFE6FFE1CFD9FFFD0EDBCF3DF0FE0E9B
:1072F000DBCF3EF0050E3D1801E13E5036E0E86878
:107300003D1802E17F0E3E182FE0030E3D1801E10B
:107310003E5028E0020E3D1801E13E5021E0010EF2
:107320003D1801E13E501AE0740E3D1801E13E5057
:1073300013E0750E3D1801E13E500CE0730E3D1850
:1073400001E13E5005E0720E3D180FE13E500DD0B8
:107350009EDF0BD09ADF09D099DF07D09DDF05D0E3
:107360009ADF03D096DF01D093DF010EE552E7CF1D
:04737000D9FF12002F
:0C7374002A0EF66E100EF76E000EF86E7A
:1073800002010900F550B36F0900F550B46F03E135
:10739000B36701D03DD00900F550AE6F0900F5503C
:1073A000AF6F0900F550B06F09000900F550E96EA4
:1073B0000900F550EA6E090009000900F550B16FA7
:1073C0000900F550B26F09000900F6CFB5F2F7CF0A
:1073D000B6F2F8CFB7F2AEC2F6FFAFC2F7FFB0C257
:1073E000F8FF0201B15302E1B25307E00900F55082
:1073F000EE6EB107F8E2B207F9D7B5C2F6FFB6C232
:10740000F7FFB7C2F8FF0201B307000EB45BBFD7A6
:02741000120068
:0E741200FE0EE3CFE9FFFF0EE3CFEAFFE9CF66
:10742000F3FFEACFF4FFFB0EE35003E1FC0EE35061
:1074300009E0FB0EE30602E2FC0EE306FD0EE3505C
:10744000EE6EF1D71200FE0EE3CFE9FFFF0EE3CFA1
:10745000EAFFF36AF46AEE5203E0F34AF42AFBD738
:107460001200FF0EE3CFF8FFE552FF0EE3CFF7FF68
:10747000E552FF0EE3CFF6FFE552E66AE66AE66AFA
:107480000900F55209E0FD0EE32A05E1FE0EE32AAC
:1074900002E1FF0EE32AF4D7FD0EE3CF3CF0FE0E2F
:0C74A000E3CF3DF0FF0EE3CF3EF0120002
:0474AC00D9CFE6FF4F
:1074B000DACFE6FFE1CFD9FFE2CFDAFFE652E652BC
:1074C000E652E652D950FB0F496EFF0EDA204A6EA3
:1074D00049C0DEFFDD6EDECFE6FFDDCFE6FFFB0E4F
:1074E000DBCFE6FFFC0EDBCFE6FFFD0EDBCFE6FFDA
:1074F000B8CEE6FFB9CEE6FFACEC2EF0496E070E33
:10750000E15C02E2E16AE552E16E4950020EF3CF1E
:10751000DBFF030EF4CFDBFF020EDBCF49F0030EDF
:10752000DBCF4AF049C0F3FF4AC0F4FF040EE15C30
:1075300002E2E16AE552E16EE552E5CFDAFFE7CF1C
:04754000D9FF12005D
:0C7544003EC048F03DC047F03D50420200
:10755000F4CF3CF0F3CF3BF03E504302F4CF3EF08B
:10756000F3CF3DF04202F3503C26F4503D22E86A4E
:107570003E2247504302F3503C26F4503D22E86A35
:107580003E2243AEC8EF3AF047503D5E48503E5A67
:1075900048AE000C42503D5E43503E5A000C3DC088
:1075A00047F03D504202F4CF3CF0F3CF3BF03E5069
:1075B0004302F4CF3EF0F3CF3DF04202F3503C26BD
:1075C000F4503D22E86A3E2247504302F3503C26E5
:0A75D000F4503D22E86A3E22000C50
:0675DA0012010002020094
:1075E0000040D80492FD820101020001090243001B
:1075F000020100C03209040000010202010005245A
:1076000000100104240202052406000105240100E3
:10761000010705810308000209040100020A0000B5
:107620000007050202400000070582024000000436
:1076300003090418035300630068006D0061006CC7
:10764000007A004800610075007300160345006968
:107650000042006F00740042006F0061007200641D
:0976600000EC752F7633764B76B1
:06766A00D9CFE6FFDACFE4
:10767000E6FFE1CFD9FFE2CFDAFFFB0EDBCF49F027
:10768000FC0EDBCF4AF00001800E4A141AE1FB0E1B
:10769000DBCFE9FFFC0EDBCFEAFFEECFF3FFEDCF50
:1076A000F4FFEE2A000EEF22F3CFE9FFF4CFEAFF5A
:1076B000FD0EDBCFEFFFEF504A6AF36E4AC0F4FFD6
:1076C00010D0FB0EDB50FE0806E1FD0EDBCFE6FF1F
:1076D0002DEC3CF005D0FD0EDBCFE6FFFEEC0EF00E
:0E76E000E552E552E5CFDAFFE7CFD9FF120001
:0276EE003B500F
:1076F0004002F3CF37F0F4CF38F04102F350382690
:10770000000EF420396E3B504202F3503926000E31
:10771000F4203A6E3B504302F3503A263C5040026C
:10772000F3503826F4503922000E3A223C504102E0
:10773000F3503926F4503A223C504202F3503A2694
:107740003D504002F3503926F4503A223D50410258
:0E775000F3503A263E504002F3503A26120003
:02775E00FF0E1C
:10776000E124E96EFF0EE220EA6EEDCFF4FFEFCFE9
:10777000F3FFF46607D0600EF36404D07B0EF36071
:1077800001D0F39A1200F36AF46AFF0EE124E96E65
:10779000FF0EE220EA6EED6607D02F0EEF6404D0F4
:0A77A0003A0EEF6001D0F32A120048
:0677AA003A6A396A386AF0
:1077B000376A200EE76ED8903B363C363D363E3673
:1077C0003736383639363A364050375C41503858BB
:1077D0004250395843503A5809E34050375E4150BF
:1077E000385A4250395A43503A5A3B2AE72EE4D786
:0277F000120085
:0E77F2004F4B0D0A000D0A0045424276313120
:10780000204542204669726D776172652056657227
:0E78100073696F6E20322E312E31640D0A0026
:02781E00C00E9A
:10782000F36E00EE00F00E0E01D81200EA6002D0F6
:0E783000EE6AFCD7F350E9601200EE6AFCD756
:02783E001DEE3D
:1078400000F02DEE00F0F86A369CBAEC39F044EC0A
:0A7850003CF016EC39F0FBD71200F3
:06785A00FF0EE350ADBA81
:1078600004D0B06AAC8EAD8A949CADA2FED7AE6E49
:06787000F36EF46A120041
:0A78760030313233343536373839FB
:0778800061626364656600AC
:027888001200EC
:02788A00FEFFFF
:04788C0000000000F8
:1078900000000000000000000000000000000000E8
:1078A00000000000000000000000000000000000D8
:1078B00000000000000000000000000000000000C8
:1078C00000000000000000000000000000000000B8
:1078D00000000000000000000000000000000000A8
:1078E0000000000000000000000000000000000098
:00000001FF
